:105C500053797374656D436C6F636B3A20384D48AC
:105C60007A000D0A00424154303A252E3266206DEA
:105C7000560D0A00424154313A252E3266206D56A7
:105C80000D0A00424154323A252E3266206D560DDF
:105C90000A00424154333A252E3266206D560D0AD1
:105CA00000424154343A252E3266206D560D0A00CA
:105CB000544F54414C3A252E3266206D560D0A0041
:105CC00054454D50303A252E326620430D0A00547B
:105CD000454D50312E303A252E326620430D0A00B4
:105CE00054454D50312E313A252E326620430D0A4F
:015CF00000B3
:0E7F5100C29CD2A08F993099FDC2A0C2992285
:1030A6001270A27BFF7A5C7950122C8E30702053FE
:1030B600B1F8C270127E00127F77127C9312787B71
:1030C6001270541272F8127ABF126410127DEC203C
:1030D6006F0302336FB2A47BFF7A5C7962122C8E87
:1030E600900285E0FCA3E0FDE4121F1D7B007A80C0
:1030F600796D7845121D72C004C005C006C00790E0
:1031060000BFE0FCA3E0FDE4121F1DA804A905AA68
:1031160006AB07D007D006D005D004121E7B90025E
:10312600BA1224847BFF7A5C7965122C8E90028712
:10313600E0FCA3E0FDE4121F1D7B007A80796D7828
:1031460045121D72C004C005C006C0079000BFE04E
:10315600FCA3E0FDE4121F1DA804A905AA06AB07FF
:10316600D007D006D005D004121E7B9002BA1224D6
:10317600847BFF7A5C7974122C8E900289E0FCA322
:10318600E0FDE4121F1D7B007A80796D7845121DE3
:1031960072C004C005C006C0079000BFE0FCA3E0F3
:1031A600FDE4121F1DA804A905AA06AB07D007D087
:1031B60006D005D004121E7B9002BA1224847BFF2F
:1031C6007A5C7983122C8E90028BE0FCA3E0FDE4FE
:1031D600121F1D7B007A80796D7845121D72C0041E
:1031E600C005C006C0079000BFE0FCA3E0FDE412E6
:1031F6001F1DA804A905AA06AB07D007D006D0054F
:10320600D004121E7B9002BA1224847BFF7A5C796A
:1032160092122C8E90028DE0FCA3E0FDE4121F1D9D
:103226007B007A80796D7845121D72C004C005C096
:1032360006C0079000BFE0FCA3E0FDE4121F1DA836
:1032460004A905AA06AB07D007D006D005D00412FC
:103256001E7B9002BA1224847BFF7A5C79A1122C21
:103266008E900289E0FEA3E0FF900288E02FFF9097
:103276000287E03EFE90028CE02FFF90028BE03E3C
:10328600FE90028EE02FFD90028DE03EFCE4121FC0
:103296001D7B007A80796D7845121D72C004C005C9
:1032A600C006C0079000BFE0FCA3E0FDE4121F1DAE
:1032B600A804A905AA06AB07D007D006D005D004F6
:1032C600121E7B9002BA1224847BFF7A5C79B012BC
:1032D6002C8E7BFF7A5C7962122C8E90029DE0FC2C
:1032E600A3E0FDE4121F1DE4FBFA79887841121D64
:1032F60072E4FBFA79C87842121E7BE4FBFA7987FE
:1033060078C3121C819002BA1224847BFF7A5C79FE
:10331600C0122C8E900299E0FCA3E0FDE4121F1D62
:103326009002BA1224847BFF7A5C79CF122C8E909D
:10333600029BE0FCA3E0FDE4121F1D9002BA1224DA
:10334600847BFF7A5C79E0122C8EC26F12255912AB
:10335600691F127D62127CEF127D0C1268564003C3
:10336600125CF1127DD71250D7127AEC127D291217
:103376006EC912526E125905900206E524F0A3E5B5
:0E33860025F0A3E522F0A3E523F00230B222E9
:107646009005367401F07E027F3C7B40E4FD127BA0
:10765600437E027F0A7B14E4127B43900224740A61
:10766600F0A374ABF0A3740AF0A374ABF0C22CC2FF
:107676002D9003FF7402F0D22ED27E90027C7450BD
:02768600F022F0
:105CF1007FFE7E01127B6D501F7B007A02E4FDFC6A
:105D0100FFFE126A9F7FFE7E03127B6D402CE4FD35
:105D1100FF7E02125EC580227FFE7E03127B6D50E4
:105D2100167B007A02E4FDFCFF7E02126A9FE4FD0D
:105D3100FFFE125EC58003D27122900000E0F520C3
:105D4100A3E0F521900238E520F0A3E521F09000D1
:105D51001A12241E90022C122484900022E0FFA328
:105D6100E0900236CFF0A3EFF0E52154072403F5CC
:105D71001364056005E513B40A04E4F51422E51380
:105D810064046005E513B409047514012275140255
:015D910022EF
:107CD100C2AFD2ACC086758640C28FD086D2AD43CA
:0E7CE100BA6043E840E4F5D843A908D2AF22C8
:107B18007580F075E18F75E9C075908075E27F75A5
:107B2800EA8075A04675E3BB75EB4675B01875E439
:0B7B3800E675EC184380C043E9802292
:1070A200E4FF127C51127B18125CF11276467D05C8
:1070B2007C007F44127A8F126980127DAB7D647FDF
:1070C200A07E0F12631212618A1261034002D25D26
:1070D2001278043007121263934002D2397E047F81
:0C70E20097125FEA4002D27B127CD122A0
:10102E00EFB4200E206603306919E4FF127C51D212
:10103E006822EFB4400D206603306907E4FF127C8E
:04104E0051D26822F1
:107C2D00D26E90049FE004F0C3940A4004E4F0D2B5
:107C3D007090049EE004F0C394C84004E4F0D26F49
:047C4D00125BAE22F6
:10774900D3EF9450EE940040037F0522D3EF943C8D
:10775900EE940040037F0422D3EF9428EE94004076
:10776900037F0322D3EF9414EE940040037F022297
:0F777900D3EF9400EE940040037F01227F0022A3
:107E140030740F9003FEE004F0C394644004E4F073
:037E2400C2742203
:106B5B00302A149003FCE004F0C3940A400BE4F0D9
:106B6B00A2B5B392B58002C2B530750D9003FDE0AE
:106B7B0004F0C394054002E4F030742C900234E02E
:106B8B00FEA3E0FF127749EF6401601CEFB402042F
:106B9B00D2A18014EFB40306D2A1D2A2800AEFB423
:0B6BAB000406D2A1D2A2D2A3127E14D5
:016BB60022BC
:1067F000C22CC22DC22E302B569003FFE07018041D
:10680000F0D22D900089E0FEA3E0FF90008CE0FD27
:1068100012631243B701229003FFE0B40116740221
:10682000F0D22E900089E0FEA3E0FF7D6412631297
:1068300043B70122E49003FFF0D22C900089E0FEE0
:10684000A3E0FF90008BE0FD12631243B70122C268
:066850002CC22DC22E2215
:107A5F00307D2CC27DE50824FE600F24F1601614E2
:107A6F006010241170191267F022D274E49003FE93
:107A7F00F022D26622B275307503C28322D28322DE
:1076C90030683CC268306924E4FF127C51D2AFC2F1
:1076D90069E490053CF07F011273D1D2ACD2ADD2EE
:1076E900CE7F70127D94127EE5127E73E490053C84
:1076F900F0A3F09003F4F09003F5F09003F6F02274
:107F0B0053B1F8C2AFD283E4FF127DC2127BBB80A8
:027F1B00EF2253
:1078ED00D283C275127E86127EF87F70127F2FC2F0
:1078FD00CE53B77E302904D2A58002C2A57F0112D6
:10790D0073D1C2AFC2ACC2ADE4F5D87F80127C5149
:06791D00D2AF127F6B22C5
:105F5C0030670E204306204403304505C267D266E5
:105F6C002230161490002AE0FF90053DE004F0C3A7
:105F7C009F406AEFF0D2662220745B202A50202BBF
:105F8C004D30191490002AE0FF90053DE004F0C359
:105F9C009F404AEFF0D26622E490053DF0A21272C7
:105FAC00107218721A721172137219721B721C729F
:105FBC00157275401390002AE0FF90053CE004F048
:105FCC009F401AEFF0D26922E490053CF022E49055
:0E5FDC00053CF0A3F022E490053CF0A3F02277
:10770900206926206623C2AFA27C727D72727268DC
:10771900724C7270726F400D90053EE06412600504
:10772900D2AF127F5FD2AF801330660AD272125283
:107739006E127F0B80063069031278ED1276C9222A
:10734100000000300062007400000089008E009986
:1073510000A200AA00BB00BF00FE00000000000068
:10736100000000000020005000820094000000A9ED
:1073710000AE00B900C200CA00DB00DF011E000040
:08738100000000000000000004
:107F1D00900402E07006C29C75995A22C29C759914
:027F2D00FF2231
:086486009005EEEEF0A3EFF02B
:10648E007B017A047900900402E02403FD127D461C
:10649E00900402E02403F582E43404F583E06F7087
:1064AE0041FF900402E0FEEFC39E502953B1F874F1
:1064BE00032FF582E43404F583E0FE9005EEE0FC54
:1064CE00A3E0F5828C83EEF09005EEE475F00112F8
:1064DE0022480F80CDD273E49005FAF0C29C7599D4
:0764EE005A22C29C7599FFC0
:0164F5002284
:1068BC00900402E0D3948C4002E4F0E4FD900402D6
:1068CC00E0FCEDC39C501D53B1F88F828E83E0FB2E
:1068DC0074032DF582E43404F583EBF00FBF000153
:1068EC000E0D80D97B017A047900EC2403FD127D16
:1068FC0046900402E02403F582E43404F583EFF0BF
:10690C00C29C9003F7E02400F582E43404F583E0A4
:02691C00F599EB
:01691E002256
:1074EF007B017A047900900402E02403FD127D46AB
:1074FF00900402E02403F582E43404F583E0B50739
:10750F001E900404E0FFB4410890053E7412F08011
:10751F0006EFB40502D267C243C29C75995A22C2C4
:05752F009C7599FF228C
:1078B6007B017A047900900402E02403FD127D46E0
:1078C600900402E02403F582E43404F583E0B5076E
:1078D60010900403E09003EFF0C243C29C75995ADE
:0778E60022C29C7599FF22EC
:1046AE00900401E0FF12250647020147020247026D
:1046BE00034702044702054702064702074702085E
:1046CE0047020947020A47130B47230C472B0D4796
:1046DE00330E473B0F471B10474311474B124753AF
:1046EE0013475B14476315476B16477317477B18C1
:1046FE0000004783EF25E02408F582E43402AF8200
:10470E00FE1268BC227E027F1E1268BC227E027FD1
:10471E00201268BC227E027F241268BC227E027F99
:10472E00261268BC227E027F281268BC227E027F7F
:10473E002A1268BC227E027F2C1268BC227E027F67
:10474E00301268BC227E027F341268BC227E027F49
:10475E00361268BC227E027F061268BC227E027F61
:10476E00081268BC227E027F381268BC227E027F4D
:10477E003A1268BC22900402E0C394804009D23AF7
:10478E009003DF7401F022900401E0B478109003DE
:10479E00EFE0B40C09D23A9003EC7401F0229004CD
:1047AE0001E0B478229003EFE025E02441F582E4A5
:1047BE003473F583E493FE740193FF9005F0EEF0ED
:1047CE00A3EFF01268BC22900401E0B479219003AB
:1047DE00EFE025E02465F582E43473F583E493FE7F
:0F47EE00740193FF9005F0EEF0A3EFF01268BC9A
:0147FD002299
:106E26007B017A047900900402E02403FD127D467A
:106E3600900402E02403F582E43404F583E06F70E5
:106E46002B900403E0FEA3E0FDEEEDFF9005DFEEE0
:106E5600F0A3EFF04E7006C29C7599FF22D27C908B
:106E660005DAE04401F0C29C75995A22C29C7599D4
:026E7600FF22F9
:10532F007B017A047900900402E02403FD127D468C
:10533F00900402E02403F582E43404F583E06F6007
:10534F00030253E6900404E0FFE4FCFDFE78101224
:10535F0023FFC004C005C006C007900403E0FFE4AC
:10536F00FCFDFE78181223FFD003D002D001D0002D
:10537F00122396C004C005C006C007900405E0FFC5
:10538F00E4FCFDFE78081223FFD003D002D001D039
:10539F0000122396A804A905AA06AB07A3E0FFE411
:1053AF00FCFDFE1223969005D61224849002A1E0F4
:1053BF007002A3E0600C9005D612241EEC4D4E4FE8
:1053CF007006C29C7599FF22D27C9005DAE04410DA
:0D53DF00F0C29C75995A22C29C7599FF225C
:107923007B017A047900900402E02403FD127D4672
:10793300900402E02403F582E43404F583E0B50700
:107943000FD27C9005DAE04420F0C29C75995A224C
:06795300C29C7599FF22A1
:107266007B017A047900900402E02403FD127D4636
:10727600900402E02403F582E43404F583E06F70A1
:1072860022D27C900403E0FEA3E0FDEEEDFF900524
:10729600DBEEF0A3EFF09005DAE04404F0C29C7553
:0972A600995A22C29C7599FF223D
:1072AF007B017A047900900402E02403FD127D46ED
:1072BF00900402E02403F582E43404F583E06F7058
:1072CF0022D27C900403E0FEA3E0FDEEEDFF9005DB
:1072DF00DDEEF0A3EFF09005DAE04408F0C29C7504
:0972EF00995A22C29C7599FF22F4
:106DD2007B017A047900900402E02403FD127D46CF
:106DE200900402E02403F582E43404F583E06F703A
:106DF2002DFF74032FF582E43404F583E0FE74E181
:106E02002FF582E43405F583EEF00FEFB407E3D2F9
:106E12007C9005DAE04480F0C29C75995A22C29CAB
:036E22007599FF60
:016E2500224A
:105B0700900401E01225065B33185B37775B537807
:105B17005B75795B3FA05B47A15B4BA25B3BA35BDC
:105B270043A45B4FAF5B97B000005BAD1274EF22ED
:105B37001278B62212532F22126E262212792322AE
:105B4700127266221272AF22126DD2229003EFE018
:105B570025E02441F582E43473F583E493FE740170
:105B670093FF9005F2EEF0A3EFF012648622900304
:105B7700EFE025E02465F582E43473F583E493FED2
:105B8700740193FF9005F2EEF0A3EFF01264862202
:105B9700900403E0B4550AD23AD238C29C75995A98
:065BA70022C29C7599FF6B
:015BAD0022D5
:10454700E49005F4F0A3F09003F7E0FFB4021A90AB
:104557000401E064A56006E49003F7F022E4900309
:10456700FAF0A3F09003F0F022900402E0FD7C0043
:104577002409FBEC33FA7E00C3EF9BEA6480F874EE
:104587008098505FED2407FDEC33FCD3EF9DEC647E
:1045970080F874809850189003F7E024FFF582E4C0
:1045A7003403F583E0FF9003FAEE8FF01222489070
:1045B70003F7E0FFB40511900404E06407700302F9
:1045C70046ADE49003F7F022EF640660030246ADC0
:1045D700900405E0640670030246AD9003F0E044E2
:1045E70020F022E49003F7F0900402E0FD2408F5A0
:1045F70082E43404F583E0FE74072DF582E4340485
:10460700F583E07C002400FFEC3EFE9003FAE06EA9
:104617007003A3E06F60079003F0E04480F090031D
:10462700F0E0FF6006900406F08007D24CE49004A7
:1046370006F0E4900402F0900405740BF090040374
:10464700E0FFA3E0900403F0A3EFF07F02900402E1
:10465700E0FE2407FDE433FCEFC39DEC6480F874AF
:104667008098501874002FF582E43404F583E0FD38
:104677009005F4E48DF01222480F80D19005F4E004
:10468700FCA3E0FF74072EF582E43404F583EFF012
:10469700ECFF900402E02408F582E43404F583EF8C
:0646A700F0C29C75995A57
:0146AD0022EA
:105E2E009003F7E02400F582E43404F583EFF0905C
:105E3E0003F7E004F0E0C3948C4002E4F09003F723
:105E4E00E064017027900400E0FF54FEB59A10EF55
:105E5E0020E006D246C2498013D249C246800D9038
:105E6E000400E0645A6005E49003F7F030460D90AC
:105E7E0003F7E0640370301246AE802B3049259054
:105E8E000402E02403FFE433FE9003F7E0D39FEE19
:105E9E006480F8748098400F125B07C249E4900347
:105EAE00F7F08003124547C243E490053CF090059D
:075EBE003DF09003F4F02217
:1059B100900400E0B45A06A3E064A56003304C44AF
:1059C100900402E02408FFE433FE9003F7E0C39F54
:1059D100EE6480F87480984014D29CE4F0C2469042
:1059E1000400F0A3F0A3F0A3F0D24380609003F78A
:1059F100E004F0C29CE02400F582E43404F583E085
:105A0100F59980499003F7E0FF6016900402E024C5
:105A110003FDE433FCC3EF9DEC6480F8748098408F
:105A210017D29CE49003F7F0C246900400F0A3F073
:105A3100A3F0A3F0D24380159003F7E004F0C29CD9
:105A4100E02400F582E43404F583E0F599E490055F
:0B5A51003CF090053DF09003F4F022C3
:107DEC009003F4E004F0C394044008E4F09003F72B
:047DFC00F0D29C2203
:107D6200305F119002B1E004F0C39405400BD25D84
:0A7D72007405F022E49002B1F02243
:0E5A5C009002BEEFF0A3EDF0A3EAF0A3EBF092
:105A6A00C24EE4A3F0305D03025AFFA3F09002BFD6
:105A7A00E0FF9002C3E0C39F507B9002C2E0FF04A4
:105A8A00F0EFC39405503E9002BEE0FD7C00900208
:105A9A00F77401F0A3F09002C0E0FFA3E09002F9CE
:105AAA00CFF0A3EFF0E4FB7F361247FE924E304E62
:105ABA0004801280C5E4F5C87F011273D1127DAB50
:105ACA001273D180B59002C2E0C3940540048025C8
:105ADA008015E49002C2F09002BEE004F09002C089
:105AEA00E475F0011222487F011273D19002C3E0DB
:0C5AFA0004F0025A77A24EB3925FA24E55
:015B0600227C
:0E671C009002C1EFF0A3EDF0A3EAF0A3EBF0C2
:10672A00C24EE4A3F0205D4D9002C5E0FF04F0EFF5
:10673A00C3940550409002C1E0FD7C00A3E09002A2
:10674A00EDF0A37401F09002C3E0FFA3E09002EF22
:10675A00CFF0A3EFF0E4FB7F36123D83924E304E2A
:10676A0004801280C3E4F5C87F011273D1127DAB95
:0C677A001273D180B3A24EB3925FA24E06
:0167860022F0
:107804007A027BA37D02E4FF12671C502E9002A330
:10781400E07004A3E060249002A7E04480F07A02C0
:107824007BA77D017F04125A5C9002A7E0547FF08D
:0C7834007A027BA77D017F04125A5C22BF
:10618A00E49002A6F0A37450F0E4A3F0A374F8F02C
:10619A00E4A3F0A3F0A37470F0A37401F0A3740352
:1061AA00F0A374FFF0E4A3F03000199002A7E044D2
:1061BA0008F09002ACE0FF9000BBE0540FFEEF4EF7
:1061CA009002ACF030013E9002A7E04404F0900245
:1061DA00ADE0FF9000BBE054F0FEEF4E9002ADF050
:1061EA009000BCE0FEA3E0FF7C007D3212252CE487
:1061FA007B257A01F9F8122304AD07AC06EC90026C
:05620A00AEF0A3EFF06F
:01620F00226C
:10610300D24D9002BD7403F09002BDE0FF14F0EF96
:1061130060727A027BA67D0B7F03125A5C505C90FF
:1061230002BC7403F09002BCE0FFD3940B504E7A90
:10613300027BBA7D0212671C9002BCE0FF7E007BEB
:106143000124A3F9EE3402FA122189FD9002BAE088
:10615300B5051374A42FF9EE3402FA122189FF90C6
:1061630002BBE06F600C9002BCE064076004C24DA8
:10617300800B9002BCE02402F080AAC24D304D880F
:0661830080028084A24DA1
:0161890022F3
:1077C7007A027BA37D02E4FF12671C502F9002A46C
:1077D700E0FF30E102D25CEF30E002D25E9002A31C
:1077E700E0FF30E307206B04D215D26DEF30E202E1
:0D77F700D2149002A4E030E20312610322DC
:107D7C007A027BB77D027F0212671C500A9002B711
:077D8C00E09002A5F0F526CE
:017D930022CD
:10691F009002B97403F09002B9E0FFD3940B50507A
:10692F007A027BB77D0212671C9002B9E0FF7E00EE
:10693F007B0124A3F9EE3402FA122189FD9002B7EC
:10694F00E0B5051374A42FF9EE3402FA122189FF72
:10695F009002B8E06F60109002B9E064076008120F
:10696F006103400CD266229002B9E02402F080A6A7
:01697F0022F5
:107BBB009002B07433F07A027BB07D017F0D125AC4
:107BCB005C50129002A7E04420F07A027BA77D0163
:067BDB007F04125A5C2237
:107DC2009002A8E054FCF04FF07A027BA87D017F7C
:057DD20005125A5C22BD
:107E27009002A7E04401F07A027BA77D017F04124C
:037E37005A5C2270
:107E3A009002A7E054FEF07A027BA77D017F04122C
:037E4A005A5C225D
:107E4D009002A7E04402F07A027BA77D017F041225
:037E5D005A5C224A
:107E60009002A7E054FDF07A027BA77D017F041207
:037E70005A5C2237
:107788009002B9EEF0A3EFF09002B9E0FEA3E07822
:1077980005CEC313CE13D8F99002AAF07A027BAAB9
:1077A8007D017F07125A5C50159002B9E0A3E09062
:0F77B80002ABF07A027BAB7D017F08125A5C2294
:107E73009002A7E04410F07A027BA77D017F0412F1
:037E83005A5C2224
:107E86009002A7E054EFF07A027BA77D017F0412EF
:037E96005A5C2211
:107E99009002A9E044F8F07A027BA97D017F0612DD
:037EA9005A5C22FE
:107EAC009002A9E05407F07A027BA97D017F0612AB
:037EBC005A5C22EB
:107EBF009002A9E044E0F07A027BA97D017F0612CF
:037ECF005A5C22D8
:107ED2009002A9E0541FF07A027BA97D017F06126D
:037EE2005A5C22C5
:107EE5009002A9E04408F07A027BA97D017F061281
:037EF5005A5C22B2
:107EF8009002A9E054F7F07A027BA97D017F06126F
:037F08005A5C229E
:107F2F009002A6E04FF07A027BA67D017F03125AE2
:027F3F005C22C2
:107D94009002A6E0FEEFF4FFEE5FF07A027BA67D90
:077DA400017F03125A5C226B
:10494500306103024A88306203024A882003030269
:104955004A88E490053AF0A3F0C3900063E095120D
:10496500900062E09511500330181ED3900065E069
:104975009512900064E09511400320180C20100951
:10498500201206201103301308C263E4900539F0A4
:1049950022C39000A3E095129000A2E09511400378
:1049A500024A81C3E5129510FFE511950FFED390DC
:1049B50000A5E09F9000A4E09E4003024A8190007C
:1049C500A6E0FEA3E0FFEE3395E0FDFC9002201289
:1049D5002437C31223B15003024A81206306900590
:1049E50039E004F09000A8E075F00AA4FF900539BD
:1049F500E0C39FE5F06480F87480985003024A880C
:104A0500AD14E5142513FFE433FEEDC39FEE64807A
:104A1500F87480985063ED25E0240AF582E43402A9
:104A2500F583E0FEA3E0C39510FFEE950FFED3904E
:104A350000A5E09F9000A4E09E503BED25E0240AF0
:104A4500F582E43402F583E0FEA3E0FF9000A2E0E6
:104A5500FAA3E0FBC3EF9BEE9A401B74017E00A80E
:104A650005088005C333CE33CED8F9FF90053AE06B
:104A75004EF0A3E04FF00D8089D26322C263E4902B
:034A85000539F000
:014A8800220B
:10795900C24D30052D20162A306527C39002B4E0A8
:1079690094B49002B3E094005011D24D900538E0E0
:1079790004F0C3940A400BD2168007C265E490054F
:0479890038F0A24DE3
:01798D0022D7
:10579800C3E5129510FFE511950FFEC3EF94B0EE27
:1057A8009404500AE5129464E51194055002D265F8
:1057B800900536E024FE605514605914606A146040
:1057C8007C2404600302585120620330637B3064F8
:1057D8001590053AE05455FFA3E054559002B7CF11
:1057E800F0A3EFF0801390053AE054AAFFA3E05429
:1057F800AA9002B7CFF0A3EFF09002B7E0FEA3E0C3
:10580800FF1277889005367402F0D261229005362F
:105818007403F0221279594030E4FFFE1277889021
:1058280005367404F0B2642212795940079005369F
:105838007405F0229005367401F0B26422900536A2
:095848007401F0C262C263C26186
:015851002234
:107BE10030052220161F900537E004F0C3942D4084
:107BF10014742DF020610EE4F0D26290053A740302
:067C0100F0A374FFF02265
:0A7F7700124945127BE112579822CF
:1079F800FFD8FFE2FFECFFF60000000A00190023A1
:107A0800002D00370041004B0055FFFBFFFCFFFD38
:107A1800FFFEFFFFFFFF000000010001000200035E
:047A28000004000551
:04380C008F828E8396
:103810007E037FE8AD82AC8312252CC006C007AEC4
:1038200083AF82C3E49FFF74109EFEAB07FAE4F9F6
:10383000F8D007D0061223049002BA122484E47F41
:103840000AFEFDFC9002BA122437D31223C7401D92
:103850009002BA12241EC3EF940AFFEE9400FEED0C
:103860009400FDEC9400FC9002BA122484904A89E2
:10387000E493FE740193FFE4FCFD9002BA12243736
:10388000C31223C7400D9002B87408F0A374B7F0B8
:103890000239F3904BC9E493FE740193FFE4FCFDFD
:1038A0009002BA122437D31223C7500D9002B87475
:1038B0000EF0A374F7F00239F390027CE09002B7A7
:1038C000F075F002904A891224DAE493FE740193B1
:1038D000FFE4FCFD9002BA122437D31223C7403B09
:1038E00090027CE0149002B7F09002B7E0FFC3941E
:1038F00000406975F002EF904A891224DAE493FEE1
:10390000740193FFE4FCFD9002BA122437D3122312
:10391000C740499002B7E014F080CE90027CE004EA
:103920009002B7F09002B7E0FFC394A0502875F062
:1039300002EF904A891224DAE493FE740193FFE4C3
:10394000FCFD9002BA122437D31223C7500890020C
:10395000B7E004F080CE9002B7E014F09002B7E038
:1039600090027CF075F002904A891224DAE493FE0A
:10397000740193FFE4FCFD9002BA12243712226B0B
:10398000E47B0AFAF9F8122279C004C005C006C027
:10399000079002B7E0FF75F002904A8B1224DAE438
:1039A00093FC740193FD75F002EF904A891224DABA
:1039B000C37401939DFFE4939CFEAB07FAE4F9F80E
:1039C000D007D006D005D004122304AB07AA069076
:1039D000027CE024CEFFE434FFFE7C007D0A12214D
:1039E000E1EF2BFFEE3ACF24ABCF340A9002B8F0D0
:0B39F000A3EFF09002B8E0FEA3E0FFA0
:0139FB0022A9
:1071D200D24D9002C0E514F0E5132514FFE433FE0E
:1071E2009002C0E0C39FEE6480F87480985028E05B
:1071F200FF25E02485F582E43402AB82FAEF25E034
:10720200240EFF7D0212671C4005C24DA24D229042
:0972120002C0E004F080C1A24DAD
:01721B002250
:10738900D24D7A027B997D027F2212671C4002C28C
:107399004D7A027B9B7D027F2412671C4002C24DFD
:1073A9007A027B9D7D027F2612671C4002C24DE551
:1073B90013D39405400F7A027B9F7D027F281267C1
:0773C9001C4002C24DA24D61
:0173D000229A
:104F22001273894003024FFF900299E0FEA3E0FF53
:104F320012380C9000C6E02FFF9000C5E03EFEC282
:104F4200AC900224F0A3EFF0D2AC90029DE0FEA35D
:104F5200E0FF7C007D1112252CE47B0AFAF9F8129D
:104F62002304EF241FFFE43EFEC2AC900228F0A30C
:104F7200EFF0D2ACE513D39405402A90029FE0FEF5
:104F8200A3E0FF7C007D1112252CE47B0AFAF9F8DC
:104F9200122304EF241FFFE43EFEC2AC90022AF06B
:104FA200A3EFF0D2AC900224E0FCA3E0FD90020259
:104FB200ECF0A3EDF0900204ECF0A3EDF0300D3D27
:104FC20090029BE0FEA3E0FF12380C9000C8E02F95
:104FD200FF9000C7E03EFEC2AC900226F0A3EFF0C5
:104FE200D2ACD3900203E09F900202E09E4006EE14
:0D4FF200F0A3EFF022900204EEF0A3EFF028
:014FFF00228F
:104BCB009002B81224A9000000009002BC1224A984
:104BDB0000000000E4900200F0A3F09002B3741701
:104BEB00F0A37470F01271D24003024D029002B721
:104BFB00E514F0E5132514FFE433FE9002B7E0FD56
:104C0B00C39FEE6480F87480984003024CD9ED2565
:104C1B00E02485F582E43402F583E0FEA3E0FF7C1B
:104C2B000E7DD812252CC006C0079000BFE0FEA356
:104C3B00E0FFFBAA06E4F9F8D007D0061223049094
:104C4B0002BC122484900200E0FEA3E0FFE4FCFD12
:104C5B009002BC122437D31223C7400E9002BC1211
:104C6B00241E900200EEF0A3EFF09002B3E0FEA33F
:104C7B00E0FFE4FCFD9002BC122437C31223C750A3
:104C8B000E9002BC12241E9002B3EEF0A3EFF020A4
:104C9B006133C2AC9002BC12241E9002B7E025E037
:104CAB00240AF582E43402F583EEF0A3EFF0D2ACE4
:104CBB009002B812241E9002BC12243712225E906E
:104CCB0002B81224849002B7E004F0024BFE20617C
:104CDB0026900200E0F511A3E0F5129002B3E0F587
:104CEB000FA3E0F510C2AC9002B812241E90021E66
:074CFB00EEF0A3EFF0D2ACD4
:014D0200228E
:10585200E49002BCF0A3F0A3F09002BEE0FFC39478
:105862000C40030258FCEF25E024F8F582E4347979
:10587200F583E493FE740193FFFBAA06EA3395E0F5
:10588200F9F89002BEE025E024FAF582E43479F5D5
:1058920083E493FE740193FFEE3395E0FDFC122244
:1058A2005EE47B02FAF9F8127602E47B0AFAF9F86E
:1058B200122279EF24ABFBEE340AFAE43DF9E43C20
:1058C200F8900228E0FEA3E0FFE4FCFDC31223B13E
:1058D200401F9002BEE025E02412F582E4347AF5FE
:1058E20083E493FF7401939002BCCFF0A3EFF080A6
:1058F200099002BEE004F002585B9002BCE0FEA3F5
:02590200E0FFC4
:015904002280
:1040EF009002B81224A9000000007A027BA17D0281
:1040FF007F2A12671C9002A1E0FEA3E0FFEE30E4DE
:10410F000944E09002A1F0A3EFF01258529000C3BF
:10411F00E0FCA3E0FDC39002A2E09DFD9002A1E0B0
:10412F009CCD2FFFED3EFE3395E0FDFC7B187AFC16
:10413F0079FF78FF122279C006C0079000C1E0FE18
:10414F00A3E0FFFBAA06EA3395E0F9F8D007D00603
:10415F0012760290027D12248490027D12241E900A
:10416F0002B2E025E025E0243CF582E43402F58339
:10417F001224849002B2E004F0C394104002E4F0E1
:10418F00E49002B7F09002B7E0FFC394105026A35B
:10419F00122437EF25E025E0243CF582E43402F5C4
:1041AF008312241E12225E9002B81224849002B74A
:1041BF00E004F080D0E47B10FAF9F89002B81224F2
:1041CF001E127602900281122484C22BC22A900002
:1041DF0028E0FEA3E0FFC3E49FFFE49EFE3395E0DB
:1041EF00FDFC900281122437C31223B15021900598
:1041FF00F7E004F0C3940A4067740AF0D22BC2AC04
:10420F0090028112241E900220122484D2AC22909C
:10421F000028E0FEA3E0FFEE3395E0FDFC90028165
:10422F00122437D31223B140299005F6E004F094FD
:10423F000A402D740AF0D22A7D647FA07E0F12638C
:10424F0012C2AC90028112241E900220122484D23A
:10425F00AC22C2AC9002201224A900000000D2AC04
:01426F00222C
:107E00001277C7C25E124BCB124F22305C05C25CA8
:047E10001240EF220B
:10664300E49002B7F0A3F0AF14E513FDE5142DFDBC
:10665300E433FCEFC39DEC6480F8748098501DEF25
:1066630025E02485F582E43402F583E0FCA3E0FD14
:106673009002B7EC8DF01222480F80CD9002B7E064
:10668300FEA3E0FF7C0E7DD812252CC006C0079028
:1066930005DFE0FEA3E0FFFBAA06E4F9F8D007D08C
:0C66A300061223049000BFEEF0A3EFF0FD
:0166AF0022C8
:107840009000C3E0FEA3E0FFC39002A2E09FFF9080
:1078500002A1E09EFE3395E0FDFC7B187AFC79FFE7
:1078600078FF1222799005D6122437127602EF4E55
:0A78700060089000C1EEF0A3EFF0F5
:01787A0022EB
:107F41009002A1E0FFA3E09000C3CFF0A3EFF022E5
:10753400900299E0FEA3E0FF12380CC39005DCE052
:107544009FFF9005DBE09EFE9000C5E0FCA3E0FDFC
:10755400C3EF9DFDEE9CFCC3ED9496EC6480948097
:107564005012ED946AEC6480947F40089000C5EE5C
:04757400F0A3EFF0A1
:0175780022F0
:1075790090029BE0FEA3E0FF12380CC39005DEE009
:107589009FFF9005DDE09EFE9000C7E0FCA3E0FDB3
:10759900C3EF9DFDEE9CFCC3ED9496EC6480948052
:1075A9005012ED946AEC6480947F40089000C7EE15
:0475B900F0A3EFF05C
:0175BD0022AB
:1075BE009005E1E0900497F09005E2E0900498F0D9
:1075CE009005E3E0900499F09005E4E090049AF0C1
:1075DE009005E5E090049BF09005E6E090049CF0A9
:1075EE009005E7E090049DF07E047F97125D92D2A5
:0475FE003AD23D221E
:106EC900307C4BC27C9005DAE030E00312664390D7
:106ED90005DAE030E4031278409005DAE030E503A2
:106EE900127F419005DAE030E2031275349005DA39
:106EF900E030E3031275799005DAE030E7031275A3
:0F6F0900BEE49005DAF0D2739005FA7402F0221C
:10705400306D0DC26DD26BE49005F9F0127E4D22B5
:10706400306B3A127D7C203134900087E075F00259
:10707400A4FFAEF09005F9E004F0C39FEE6480F83D
:107084007480984018C26BE4F0127E60307902C2BA
:0E70940019C21BC21C301505C2151278042249
:1072F800306C0DC26CD26AE49005F8F0127E272239
:10730800306A35127D7C20302F900087E075F002BE
:10731800A4FFAEF09005F8E004F0C39FEE6480F897
:107328007480984013C26AE4F0127E3A307807C23B
:0973380018C214127804C21A22D2
:107CEF00300719303B119003E4E004F0C3940540D2
:0D7CFF000BD2397405F022E49003E4F0226A
:1069E1009002E1EEF0A3EFF0A3EDF0A3EAF0A3EB48
:0169F100F0B5
:1069F200C24D203941E4A3F09002E1E0FCA3E0FDA6
:106A0200A3E09002F7F0E4A3F09002E4E0FFA3E039
:106A12009002F9CFF0A3EFF07B017FA01247FE5066
:106A220004D24D80117F011273D19002E6E004F08E
:0D6A3200E0C3940540C2A24DB3923BA24DBB
:016A3F002234
:106A40009002C3EEF0A3EFF0A3EDF0A3EAF0A3EB06
:016A5000F055
:106A5100C24E203941E4A3F09002C3E0FCA3E0FD63
:106A6100A3E09002EDF0E4A3F09002C6E0FFA3E002
:106A71009002EFCFF0A3EFF07B017FA0123D835096
:106A810004D24E80117F011273D19002C8E004F04C
:0D6A9100E0C3940540C2A24EB3923BA24E5A
:016A9E0022D5
:1066B0007E027FBA7B08E4FD127B43E49002B8F0CF
:1066C000A3F09002B8E0FEA3E0FFE4FCFD7BFF7ABC
:1066D00007F9F8D31223B1402E53B1F89002B8E075
:1066E000FEA3E07805C333CE33CED8F9241FFFE4F0
:1066F0003EFE7A027BBA7D011269E19002B8E47530
:10670000F00112224880BB7A027BBA7D087FE07ECE
:0B671000FF1269E1E49003DDF0A3F04C
:01671B00225B
:10639300C24D7A027BB77D087FE07EFF126A40928E
:1063A3004D9002B8E0FF9002B7E02F9002B9F09051
:1063B30002BCE0FF9002BBE02F9002BDF09002BA56
:1063C300E0FF9002B9E0B507179002B7E0FEA3E043
:1063D3007C002400FFEC3E9003DDF0A3EFF0802A65
:1063E3009002BEE0FF9002BDE0B507179002BBE04C
:1063F300FEA3E07C002400FFEC3E9003DDF0A3EF5E
:0C640300F08007E49003DDF0A3F0A24D50
:01640F00226A
:1070EE00E49002C1F07E047F97123BC17E047F972D
:1070FE007C027DB87B07127A2CE4FF74B82FF582E0
:10710E00E43402F583E0FE9002C1E02EF00FEFB4FE
:10711E0007E99002C1E09002BFF0A3745AF07A0220
:0B712E007BB87D097FF07EFF1269E155
:017139002233
:107688009003DDE0FCA3E0FDEC9002D9F0AF05A388
:10769800EFF09002D9E02F9002DCF09002D9E09050
:1076A80002DDF09002DAE09002DEF09002DCE09079
:1076B80002E0F07A027BD97D087FE07EFF1269E163
:0176C800229F
:053F3C009002B8EFF057
:103F41006410701A7E037FE57C027DB97B03127ACF
:103F51002C7E037FE97C027DBC127A2C801F7E04BB
:103F61007F97123BC17E047F977C027DB97B031250
:103F71007A2C7E047F9A7C027DBC127A2C900206F8
:103F8100E0FCA3E0FDEC9002BFF0A3EDF09002088D
:103F9100E0FCA3E0FDEC9002C1F0A3EDF090022C57
:103FA10012241E78181223D89002C3EFF090022C2D
:103FB10012241E78101223D89002C4EFF090022C24
:103FC10012241E78081223D89002C5EFF090022C1B
:103FD10012241E9002C6EFF090023012241E7818AF
:103FE1001223D89002C7EFF090023012241E7810ED
:103FF1001223D89002C8EFF090023012241E7808E4
:104001001223D89002C9EFF090023012241E9002C0
:10401100CAEFF090021EE0FCA3E0FDAE047818CEDA
:10402100C313CE13D8F99002CBF0EDAE047810CEC5
:10403100C313CE13D8F99002CCF090021EE0FCA37A
:10404100E0FDEC9002CDF0A3EDF090022012241ED1
:1040510078181223EB9002CFEFF090022012241E69
:1040610078101223EB9002D0EFF090022012241E60
:1040710078081223EB9002D1EFF090022012241E57
:104081009002D2EFF0900224E0FCA3E0FDEC90025C
:10409100D3F0A3EDF0900236E0FCA3E0FDEC90023A
:1040A100D5F0A3EDF09002B8E09002D7F0A3745AD6
:1040B100F09003DDE0FEA3E0FF7A027BB97D2012E0
:1040C10069E19003DDE475F0201222489003DDE000
:1040D100FEA3E0FFE4FCFD7BE07AFFF9F8D31223B5
:0D40E100B15007E49003DDF0A3F0127688E3
:0140EE0022AF
:106787009003EFE02480FFE434FFEF7D00C454F072
:10679700FC900401E02488FFE434FFFEEF7807C390
:1067A70033CE33CED8F92DFFEE3CFE900402E0FD48
:1067B7007A047B03126A407B017A04790090040211
:1067C700E02403FD127D46900402E02403F582E4F1
:1067D7003404F583EFF0C29C9003F7E02400F582C0
:0867E700E43404F583E0F599A8
:0167EF002287
:1064F6009003EFE02480FFE434FFEF7D00C454F006
:10650600FC9004A1E02488FFE434FFFEEF7807C383
:1065160033CE33CED8F92DFFEE3CFE9004A2E0FD3B
:106526007A047BA3126A407B017A0479A09004A2C4
:10653600E02403FD127D469004A2E024A3F582E444
:106546003404F583EFF0758640C2A49003F8E02486
:0E655600A0F582E43404F583E0F5A1E4F586B7
:016564002214
:106565009003EFE02480FFE434FFEF7D00C454F096
:10657500FC900541E02488FFE434FFFEEF7807C373
:1065850033CE33CED8F92DFFEE3CFE900542E0FD2B
:106595007A057B43126A407B017A05794090054272
:1065A500E02403FD127D46900542E02443F582E494
:1065B5003405F583EFF0758640C2949003F9E02425
:0E65C50040F582E43405F583E0F591E4F586B7
:0165D30022A5
:1074A9007E047F97123BC17E047F977C047D037B1A
:1074B90007127A2C7B017A047900900402E02403F4
:1074C900FD127D46900402E02403F582E43404F5BC
:1074D90083EFF0C29C9003F7E02400F582E43404C2
:0674E900F583E0F5992295
:10713A007E047F97123BC17E047F977C047DA37BEC
:10714A0007127A2C7B017A0479A09004A2E0240326
:10715A00FD127D469004A2E024A3F582E43404F5EE
:10716A0083EFF0758640C2A49003F8E024A0F5826C
:0C717A00E43404F583E0F5A1E4F586227E
:107186007E047F97123BC17E047F977C057D437BFF
:1071960007127A2C7B017A057940900542E0240398
:1071A600FD127D46900542E02443F582E43405F560
:1071B60083EFF0758640C2949003F9E02440F5828F
:0C71C600E43405F583E0F591E4F5862241
:105905002007030259B0203A030259B0C23A303891
:1059150005C2381266B09003DFE0FF7008A3E0709F
:1059250004A3E06021EF6008E49003DFF0126787CD
:105935009003E0E06005E4F01265659003E1E06046
:1059450005E4F01265659003ECE0FF7008A3E070D4
:1059550004A3E06021EF6008E49003ECF01274A961
:105965009003EDE06005E4F012713A9003EEE0601B
:1059750005E4F0127186303D05C23D1270EE303CF3
:105985000CC23C9002B77410F0FF123F3C30420C41
:10599500C2429002B77401F0FF123F3C303F0CC287
:0B59A5003F9002B77402F0FF123F3C7D
:0159B00022D4
:1050D7002007030251A990002EE0FF9003DAE004B5
:1050E700F0C39F4009E4F07E047F97123BC1900311
:1050F700DBE475F001122248FEC3E5F09410EE944C
:105107000E400BE49003DBF0A3F0D23AD23D202A05
:105117001ED241304006C240D23AD24230190B303B
:105127003E08C23ED23AD23F8005201902D23E3015
:10513700416990002CE0FEA3E0FFEE3395E0FDFC13
:10514700900220122437C31223B1404F9003E2E0AC
:105157007002A3E070147E047F97123BC17E047F28
:10516700977C037DE57B07127A2C90002BE0FF7E6E
:10517700007C007D3C1221E19003E2E475F001120E
:105187002248FCD3E5F09FEC9E4017E49003E2F041
:10519700A3F0D240C241D23AD23C22E49003E2F0DB
:0351A700A3F02250
:031053000265D45F
:1065D400C0E0C083C082C0D075D000C007C086753B
:1065E400860030D807C2D87F0112102E30D907C2D6
:1065F400D97F0212102E30DA07C2DA7F0412102E6D
:1066040030DB07C2DB7F0812102E30DC07C2DC7FD0
:106614001012102E30DD07C2DD7F2012102E30DE66
:1066240007C2DE7F4012102E30DF07C2DF7F8012E8
:0F663400102ED086D007D0D0D082D083D0E032C5
:03102B00021003AD
:10100300C0E0C083C082C0D0C086758640C28F75E1
:101013008600127C2DD086D0D0D082D083D0E0320F
:105BAE00307D03025C4F75090F20A7057509018032
:105BBE000620B003750902E509650C6038050EE58F
:105BCE000E7002050DC3E50B940AE50A94004065BC
:105BDE00E50E940AE50D94004067E50B9490E50AF6
:105BEE0094014008E50C4440F5088003850C08D26A
:105BFE007D80428040E509640F6037E4F50DF50EB7
:105C0E00050BE50B7002050AB4900EE50AB4010906
:105C1E00E50C4410F508D27D22E50BB4B023E50A5D
:105C2E00B4041E750A01750B90E50C4420F508D2DC
:105C3E007D2275080FE4F50AF50BF50DF50E8509B5
:015C4E000C49
:015C4F002232
:10798E00AB07AA06C2AF43A701EAF5F7AF038FFB19
:10799E00AF058FFC75F26E75F30575F40A75F50972
:1079AE00EAADF7B50509E475F606000000000053D0
:0579BE00A7FED2AF227C
:107C0700D250E4FDFCEF2DFBEE3C8B82F583E49331
:107C17006004C250800D0DBD00010CE4B505E6EC13
:057C2700B402E2A250CE
:017C2C002235
:086C6D009002BDEEF0A3EFF070
:106C7500D250AE04AF05E4A3F0A3F09002BFE0FC50
:106C8500A3E0FDC3EC940250369002BEE02DFD90CA
:106C950002BDE03C8D82F583E493FD9002BFE0FAEE
:106CA500A3E02FF582EE3AF583E0FCED6C6004C2BB
:106CB50050800C9002BFE475F00112224880BCA2FE
:016CC500507E
:016CC60022AB
:086077009002BDEEF0A3EFF072
:10607F00C250AF05A3ECF0A3EFF0E4FDFC9002BD1E
:10608F00E0FAA3E0FB2DF5FBEB2DEA3CF5F7A3E0DF
:10609F00FEA3E02DF582EE3CF583E0F5FC75F26E84
:1060AF0020AF3D75F305E5A7603275F40A9005FB47
:1060BF00E06455702375F5099002BEE02D9002BD86
:1060CF00E03CABF7B5030DE475F6060000000000E9
:1060DF00D2508010C2508019C2508015C25080110A
:1060EF00C250800D0DBD00010CED7003EC64027009
:0360FF008CA25020
:01610200227A
:0E5EC5009002B9EEF0A3EFF0A3ECF0A3EDF025
:105ED300C24F53B1F8C2AF43A7019002B9E0FF7EAE
:105EE30000F5F775F2E620AF5B75F305E5A760549F
:105EF30075F40A9005FBE06455704975F509ADF733
:105F0300EF6D7001EE703D75F60600000000009025
:105F130002B9E0FEA3E0FF127C0750289002B9E02B
:105F2300FEA3E0FFA3E0FCA3E0FD12607750159011
:105F330002B9E0FEA3E0FFA3E0FCA3E0FD126C6D59
:105F43005002D24FE4F5F2F5F3F5F4F5F5F5F65317
:085F5300A7FEF5F7D2AFA24F43
:015F5B002223
:10526E00C24DC24E20720302532EC2729005FB74C1
:10527E0055F0E513D39405400C9002B77427F0A3B4
:10528E007410F0800A9002B77413F0A37488F09033
:10529E0002B7E0FEA3E0FFC390021FE09F90021E44
:1052AE00E09E406B9001FEE0645A7004A3E064A59A
:1052BE00705DFDFCFFFE125EC54023E4FDFCFFFEAB
:1052CE00125EC54019D24D74FF9001FEF0A3F0FDA1
:1052DE007FFE7E0112798E7DFF7FFF12798EE4FDB7
:1052EE00FCFF7E02125EC5402AE4FDFCFF7E021228
:1052FE005EC5401FD24E74FF9001FEF0A3F0FD7FFD
:10530E00FE7E0312798E7DFF7FFF12798E8004D28E
:10531E004DD24EE49005FBF0304D05304E02D27169
:01532E00225C
:0E6A9F009002B7EEF0A3EFF0A3EAF0A3EBF045
:106AAD00D24DAE04AF058E158F16C2AF43A701535D
:106ABD00B1F8E4FFFED39002BAE09F9002B9E09ED8
:106ACD0040279002B8E02FFD9002B7E03E8D82F591
:106ADD0083E493851682851583F00516E5167002FD
:106AED0005150FBF00010E80CC53A7FED2AFA24DEE
:016AFD002276
:107DD7003073119005FAE004F0C394024006C273B1
:057DE700E4F0D272225D
:107B6D00C24D43A701EEC313FEEF1325E0FFEE3325
:107B7D008F82F583740193B4A507E493B45A02D2AE
:067B8D004D53A7FEA24DBE
:017B930022CF
:057A8F009002B7EFF0CA
:107A9400758640758830AE04AF057C1F7D40122585
:107AA4002CE4FB7A01F9F8122304C3E49FFFE49E5B
:0A7AB400FE8F8CF58DD28AE4F58672
:017ABE0022A5
:057C51009002B7EFF006
:107C5600A2AFE433FFC2AF43B20800000000000049
:0C7C6600000053B26043B20424FF92AF50
:017C720022EF
:106210009005E8EEF0A3EFF0A3EDF075C7B09005A0
:10622000E8E0FEA3E0FFFBAA06E4F9F87FD87EB819
:106230007D05FC1276028FCC9005E8E0FEA3E0FF1E
:10624000FBAA06E4F9F87FD87EB87D05FC12760239
:1062500078081223EB8FCDAFCDEFFEADCC7C00E400
:106260002DFFEC3EFE9005EAE0FBFD1221E17D648E
:106270001221F38FCEAFCDEFFEADCC7C00E42DFF2D
:10628000EC3EFEAD031221E17D641221F3EEF5CF69
:0162900022EB
:106291009005EBEEF0A3EFF0A3EDF075B6B090052D
:1062A100EBE0FEA3E0FFFBAA06E4F9F87FD87EB895
:1062B1007D05FC1276028FAE9005EBE0FEA3E0FFB8
:1062C100FBAA06E4F9F87FD87EB87D05FC127602B8
:1062D10078081223EB8FAFAFAFEFFEADAE7C00E4D9
:1062E1002DFFEC3EFE9005EDE0FBFD1221E17D640A
:1062F1001221F38FA4AFAFEFFEADAE7C00E42DFF12
:10630100EC3EFEAD031221E17D641221F3EEF5A511
:016311002269
:106312009002BCEEF0A3EFF0A3EDF075B7B09002DF
:10632200BCE0FEA3E0FFFBAA06E4F9F87FD87EB842
:106332007D05FC1276028FBC9002BCE0FEA3E0FF5A
:10634200FBAA06E4F9F87FD87EB87D05FC12760236
:1063520078081223EB8FBDAFBDEFFEADBC7C00E42D
:106362002DFFEC3EFE9002BEE0FBFD1221E17D64BA
:106372001221F38FBEAFBDEFFEADBC7C00E42DFF5A
:10638200EC3EFEAD031221E17D641221F3EEF5BF76
:0163920022E8
:1073D100E5B2547070067C067D868020E5B254705B
:1073E100FEBE20067C037D438012E5B25470FEBED2
:1073F10040067C017DA180047C007D8BE4FEEEC310
:107401009F5014E4FBFAC3EB9DEA9C50070BBB00B1
:07741100010A80F20E80E782
:017418002251
:1068560090002FE0645A705A900061E0645A7052BA
:10686600900073E0645A704A900088E0645A70425F
:1068760090008DE0645A703A900098E0645A703245
:106886009000A1E0645A702A9000A9E0B45A2390BF
:1068960000BAE0B45A1C9000BEE0B45A159000CA83
:1068A600E0B45A0E9001FEE0645A7004A3E064A5B9
:0668B6006002C322D322A0
:087B43009002C3EEF0A3EFF085
:107B4B00E4FFEFC39B501A9002C3E0F8A3E0F58269
:107B5B008883EDF09002C3E475F0011222480F8088
:017B6B00E138
:017B6C0022F6
:087A2C009002D9EEF0A3EFF087
:107A3400E4FFEFC39B50239002D9E0F8A3E0F58262
:107A44008883E08D828C83F00DBD00010C9002D9F7
:0A7A5400E475F0011222480F80D8FB
:017A5E002205
:0C7F5F00758E55438701000000000022D1
:0C7F6B00758E55438702000000000022C4
:107AEC0090053EE064127023204306204403304589
:107AFC001A207317207214C2AFE4F5A8F5A9F58803
:0C7B0C00F5E8F59DF59CF59812000022AC
:10721C00D228D229201403301602C22820110F20A4
:10722C00130C201B09201C06201503301602C22942
:10723C00202B0E201009201206201803301A02C22F
:10724C0028202A05301902C229201B06201C0330D5
:0A725C001502C228301A02C22922CE
:107ABF0012721CA276302801B34008A27730290138
:107ACF00B35019A2289276A2299277A229E433FF04
:0D7ADF0025E0FFA228E4334FFF127DC222F4
:10741900201844C3900063E09512900062E0951132
:10742900501F9003BCE475F001122248FEC3E5F039
:107439009401EE94004020D218E49003BCF0A3F02C
:1074490022D3900065E09512900064E09511400701
:08745900E49003BCF0A3F02253
:10746100201944D3900075E09510900074E0950FB9
:10747100401F9003BEE475F001122248FEC3E5F0FF
:107481009401EE94004020D219E49003BEF0A3F0E1
:1074910022C3900077E09510900076E0950F500799
:0874A100E49003BEF0A3F02209
:106F180020104B90008EE0FEA3E0FF900204E0FCFE
:106F2800A3E0FDD39FEC9E401F9003CEE475F001D3
:106F3800122248FEC3E5F09401EE94004020D210DE
:106F4800E49003CEF0A3F022900090E0FEA3E0FFCF
:0F6F5800C3ED9FEC9E5007E49003CEF0A3F02210
:106F670020124B900092E0FEA3E0FF900202E0FCAB
:106F7700A3E0FDC39FEC9E501F9003D2E475F00180
:106F8700122248FEC3E5F09401EE94004020D2128D
:106F9700E49003D2F0A3F022900094E0FEA3E0FF78
:0F6FA700D3ED9FEC9E4007E49003D2F0A3F022BD
:106FB60020114B900099E0FEA3E0FF900204E0FC54
:106FC600A3E0FDD39FEC9E401F9003D0E475F00133
:106FD600122248FEC3E5F09401EE94004020D2113F
:106FE600E49003D0F0A3F02290009BE0FEA3E0FF24
:0F6FF600C3ED9FEC9E5007E49003D0F0A3F02270
:1070050020134B90009DE0FEA3E0FF900202E0FC00
:10701500A3E0FDC39FEC9E501F9003D4E475F001DF
:10702500122248FEC3E5F09401EE94004020D213ED
:10703500E49003D4F0A3F02290009FE0FEA3E0FFCC
:0F704500D3ED9FEC9E4007E49003D4F0A3F0221C
:10787B00307E37124BCB124F2212741912746112D5
:10788B006F18126F67126FB612700590053FE00408
:10789B00F0C394024014C27E205D09203906207B80
:0B78AB0003307103D266221243DF227B
:1051AA0020185C201459C3900063E09512900062A5
:1051BA00E095115033900066E075F00AA4FFAEF056
:1051CA009003BCE475F001122248FCC3E5F09FECA1
:1051DA009E500302526DD218C278E49003BCF0A329
:1051EA00F09003D6F0A3F022D3900065E0951290D8
:1051FA000064E09511406CE49003BCF0A3F0222017
:10520A007861D3900065E09512900064E0951140B2
:10521A003C900067E075F00AA4FFAEF09003D6E474
:10522A0075F001122248FCC3E5F09FEC9E40343031
:10523A000E06D278D26C8007C218C214127804E41F
:10524A009003BCF0A3F09003D6F0A3F022C3900021
:10525A0063E09512900062E095115007E49003D63E
:04526A00F0A3F0229B
:1053EC00201959D3900075E09510900074E0950F3A
:1053FC004033900078E075F00AA4FFAEF09003BE45
:10540C00E475F001122248FCC3E5F09FEC9E5003BA
:10541C000254A7D219C279E49003BEF0A3F0900312
:10542C00D8F0A3F022C3900077E09510900076E0BE
:10543C00950F5067E49003BEF0A3F02220795CC373
:10544C00900077E09510900076E0950F5037900023
:10545C0079E075F00AA4FFAEF09003D8E475F00182
:10546C00122248FCC3E5F09FEC9E402F300F06D271
:10547C0079D26D8002C219E49003BEF0A3F09003C0
:10548C00D8F0A3F022D3900075E09510900074E052
:0C549C00950F4007E49003D8F0A3F02225
:1054A80020105E90008EE0FEA3E0FF900204E0FC76
:1054B800A3E0FDD39FEC9E4031900096E075F01478
:1054C800A4FFAEF09003CEE475F001122248FAC3AF
:1054D800E5F09FEA9E5003025563D210E49003CE94
:1054E800F0A3F09003C0F0A3F022900090E0FEA398
:1054F800E0FFC3ED9FEC9E5062E49003CEF0A3F072
:1055080022900090E0FEA3E0FF900204E0FCA3E0FC
:10551800FDC39FEC9E502E900096E075F014A4FFFA
:10552800AEF09003C0E475F001122248FAC3E5F02A
:105538009FEA9E4026C210E49003CEF0A3F09003A9
:10554800C0F0A3F02290008EE0FEA3E0FFD3ED9F11
:0C555800EC9E4007E49003C0F0A3F0229A
:1055640020125E900092E0FEA3E0FF900202E0FCB5
:10557400A3E0FDC39FEC9E5031900096E075F014BB
:10558400A4FFAEF09003D2E475F001122248FAC3EE
:10559400E5F09FEA9E500302561FD212E49003D214
:1055A400F0A3F09003C4F0A3F022900094E0FEA3D3
:1055B400E0FFD3ED9FEC9E4062E49003D2F0A3F0B1
:1055C40022900094E0FEA3E0FF900202E0FCA3E03E
:1055D400FDD39FEC9E402E900096E075F014A4FF3E
:1055E400AEF09003C4E475F001122248FAC3E5F06A
:1055F4009FEA9E4026C212E49003D2F0A3F09003E7
:10560400C4F0A3F022900092E0FEA3E0FFC3ED9F5C
:0C561400EC9E5007E49003C4F0A3F022C9
:1056200020115E900099E0FEA3E0FF900204E0FCF0
:10563000A3E0FDD39FEC9E4031900096E075F014FE
:10564000A4FFAEF09003D0E475F001122248FAC333
:10565000E5F09FEA9E50030256DBD211E49003D09E
:10566000F0A3F09003C2F0A3F02290009BE0FEA311
:10567000E0FFC3ED9FEC9E5062E49003D0F0A3F0F6
:105680002290009BE0FEA3E0FF900204E0FCA3E078
:10569000FDC39FEC9E502E900096E075F014A4FF81
:1056A000AEF09003C2E475F001122248FAC3E5F0AF
:1056B0009FEA9E4026C211E49003D0F0A3F090032D
:1056C000C2F0A3F022900099E0FEA3E0FFD3ED9F8B
:0C56D000EC9E4007E49003C2F0A3F0221F
:1056DC0020135E90009DE0FEA3E0FF900202E0FC30
:1056EC00A3E0FDC39FEC9E5031900096E075F01442
:1056FC00A4FFAEF09003D4E475F001122248FAC373
:10570C00E5F09FEA9E5003025797D213E49003D41E
:10571C00F0A3F09003C6F0A3F02290009FE0FEA34C
:10572C00E0FFD3ED9FEC9E4062E49003D4F0A3F035
:10573C002290009FE0FEA3E0FF900202E0FCA3E0B9
:10574C00FDD39FEC9E402E900096E075F014A4FFC4
:10575C00AEF09003C6E475F001122248FAC3E5F0EE
:10576C009FEA9E4026C213E49003D4F0A3F090036A
:10577C00C6F0A3F02290009DE0FEA3E0FFC3ED9FD6
:0C578C00EC9E5007E49003C6F0A3F0224E
:106CC700201A5590006D12241E90027D122437D38E
:106CD7001223B1402A900071E075F00AA4FFAEF0CC
:106CE7009003CAE475F001122248FCC3E5F09FEC5B
:106CF7009E4025D21AD26CE49003CAF0A3F022205A
:106D07006A16D39003CBE094009003CAE094004046
:096D17000774FFF5F01222482276
:106D2000201B5590007D12241E90027D122437C333
:106D30001223B1502A900081E075F00AA4FFAEF052
:106D40009003B8E475F001122248FCC3E5F09FEC13
:106D50009E4025E49003B8F0A3F0D21BD26D222010
:106D60006B16D39003B9E094009003B8E094004010
:096D70000774FFF5F0122248221D
:106D7900201C5590008212241E90027D122437C3D4
:106D89001223B1502A900086E075F002A4FFAEF0FC
:106D99009003BAE475F001122248FCD3E5F09FECA8
:106DA9009E4025E49003BAF0A3F0D21CD26D2220B4
:106DB9006B16D39003BBE094009003BAE0940040B3
:096DC9000774FFF5F012224822C4
:107C9300207E1B1251AA1253EC1254A812556412DF
:0F7CA30056201256DC126CC7126D20126D79221A
:10641000300272201B06201C03301539900072E0F8
:1064200075F014A4FFAEF09003CCE475F0011222D5
:1064300048FCC3E5F09FEC9E401BE49005F9F0900A
:1064400003CCF0A3F0C21BC21CC26DC26B30150599
:10645000C215127804301A2D900072E075F014A461
:10646000FFAEF09003C8E475F001122248FCD3E5BA
:10647000F09FEC9E400FE49003C8F0A3F0C21A9086
:0664800005F8F0C26A22DB
:107D0C00300719307A11900496E004F0C3940540C2
:0D7D1C000BD27B7405F022E4900496F02257
:0E6BB7009002EEEFF0A3EDF0A3EAF0A3EBF0F6
:106BC500C250207B40E4A3F09002EEE0FD7C00A3E0
:106BD500E09002F7F0E4A3F09002F0E0FFA3E0906C
:106BE50002F9CFF0A3EFF0E4FB7FDE1247FE50047D
:106BF500D25080117F011273D19002F2E004F0E0CF
:0C6C0500C3940540C3A250B3927AA25081
:016C11002260
:0E6C12009002E4EFF0A3EDF0A3EAF0A3EBF0A4
:106C2000C24F207B40E4A3F09002E4E0FD7C00A38F
:106C3000E09002EDF0E4A3F09002E6E0FFA3E09024
:106C400002EFCFF0A3EFF0E4FB7FDE123D835004B0
:106C5000D24F80117F011273D19002E8E004F0E07E
:0C6C6000C3940540C3A24FB3927AA24F28
:016C6C002205
:083BC1009002D9EEF0A3EFF031
:103BC900C24E7A027BDB7D09E4FF126C12400302CC
:103BD9003D809002E2E030E003023D739002DDE0B7
:103BE90020E703023C929002DBE0FF5470945040BE
:103BF90003023C92EF540F94094003023C92E054B3
:103C09007F94594003023C92A3E0FF5470945050B2
:103C190078EF540F94095071E0547F9459506AA376
:103C2900E0FF543094205061EF540F9409505AE04A
:103C3900542F94245053A3E0FF54309430504AEF4A
:103C4900540F94095043E0543FFF9431503BEF60C7
:103C590038A3E0FF54109410502FEF540F940950DB
:103C690028E0541FFF94125020EF601DA3E0FF5479
:103C7900F094905014EF540F9409500DE09499501A
:103C890008A3E05407940640779002D9E0FEA3E028
:103C9900FFF5828E83E09002DBF08F828E83A3E0B2
:103CA9009002DCF09002D9E0A3E0F5828E83A3A311
:103CB900E09002DDF08F828E83A3A3A3E09002DE61
:103CC900F09002D9E0A3E02404F582E43EF583E014
:103CD9009002DFF0EF2405F582E43EF583E09002DF
:103CE900E0F09002D9E0A3E02406F582E43EF583F2
:103CF900E09002E1F07E027FDB125D92924E8077C6
:103D09009002DBE0FF9002D9E0FCA3E0FDF5828C94
:103D190083EFF09002DCE08D828C83A3F09002DDCA
:103D2900E0541F8D828C83A3A3F09002DEE08D8284
:103D39008C83A3A3A3F09002DFE0FFED2404F582B6
:103D4900E43CF583EFF09002E0E0FFED2405F58215
:103D5900E43CF583EFF09002E1E0FFED2406F58203
:103D6900E43CF583EFF0D24E800D9002D9E0FEA33A
:093D7900E0FF125D92924EA24E91
:013D8200221E
:085D92009002E4EEF0A3EFF033
:105D9A00C24FA37490F07A027BE67D017F07126BF3
:105DAA00B7924F9002E4E0FEA3E0FFF5828E83E013
:105DBA009002E7F08F828E83A3E09002E8F09002CF
:105DCA00E4E0FCA3E0FDF5828C83A3A3E044809089
:105DDA0002E9F08D828C83A3A3A3E09002EAF090FB
:105DEA0002E4E0A3E0FF2404F582E43EF583E090B8
:105DFA0002EBF0EF2405F582E43EF583E09002EC35
:105E0A00F09002E4E0A3E02406F582E43EF583E0A4
:105E1A009002EDF07A027BE77D07E4FF126BB792FE
:035E2A004FA24F35
:015E2D002252
:085FEA009002B7EEF0A3EFF006
:105FF200C24DE49002C2F07E027FB97B09FD127BA2
:10600200437A027BB97D097FF07EFF126A40E4FF8A
:1060120074B92FF582E43402F583E0FE9002C2E007
:106022002EF00FEFB407E99002C2E0FF9002C0E049
:10603200B50706A3E0645A601BE49002B9F0A3F02E
:10604200A37412F0A37401F0A37405F0A37420F0FA
:10605200A37405F07E027FB99002B7E0FCA3E0FDD5
:106062007B07127A2C9002B7E0FEA3E0FF123BC13D
:04607200924DA24D5C
:016076002207
:104E220000070E091C1B1215383F363124232A2D88
:104E320070777E796C6B6265484F464154535A5D78
:104E4200E0E7EEE9FCFBF2F5D8DFD6D1C4C3CACD68
:104E520090979E998C8B8285A8AFA6A1B4B3BABD58
:104E6200C7C0C9CEDBDCD5D2FFF8F1F6E3E4EDEA48
:104E7200B7B0B9BEABACA5A28F88818693949D9A38
:104E82002720292E3B3C35321F18111603040D0A28
:104E92005750595E4B4C45426F68616673747D7A18
:104EA200898E878095929B9CB1B6BFB8ADAAA3A408
:104EB200F9FEF7F0E5E2EBECC1C6CFC8DDDAD3D4F8
:104EC200696E676075727B7C51565F584D4A4344E8
:104ED200191E171005020B0C21262F283D3A3334D8
:104EE2004E49404752555C5B7671787F6A6D6463C8
:104EF2003E39303722252C2B0601080F1A1D1413B8
:104F0200AEA9A0A7B2B5BCBB9691989F8A8D8483A7
:104F1200DED9D0D7C2C5CCCBE6E1E8EFFAFDF4F397
:107D4600E4FFEDD3940040131221896F904E2293E5
:0B7D5600FF740129F9E43AFA1D80E7F0
:017D610022FF
:107B9400D2527D807CBBE5C820E31053B1F8ED4C94
:107BA4006009ED1D70011C80ED80EBE5D154F86F88
:067BB4006002C252A25261
:017BBA0022A8
:1047FE009002F6EBF09002F3EFF0A3ECF0A3EDF0E5
:10480E00D2519002FF74BBF0A37480F09002FBEFC4
:10481E00F0A3EDF09002F9E0FEA3E0F5828E83E0C6
:10482E009002FDF07B017A0279FB7D03127D4690AA
:10483E0002FEEFF09002F7E0D394005003024942DB
:10484E0043E6C043D10143C80175C8607F08127B9F
:10485E0094400C7F10127B944005C25102491F9068
:10486E0002F3E0F58D75C8407F18127B944005C2A7
:10487E005102491F9002F6E0B401159002F4E0F5E2
:10488E008D75C8407F28127B944005C25102491F86
:10489E009002F4E0A3E0F58D75C8407F28127B945A
:1048AE004004C251806B9002F8E06401702EA3E0C8
:1048BE00FEA3E0F5828E83E0F58D75C8407F281249
:1048CE007B944004C25180499002FEE0F58D75C87C
:1048DE00407F28127B944039C2518035E4FE90020D
:1048EE00F7E0FFEEC39F50299002F9E0FCA3E0F53C
:1048FE00828C83E0F58D75C8407F28127B9440042E
:10490E00C251800D9002F9E475F0011222480E801A
:10491E00CD75C850E5C830E41B53B1F89002FFE0E6
:10492E007002A3E0600E9002FF74FFF5F0122248B1
:06493E0080E280E0A251BE
:014944002250
:0A3D8300AA079002EAECF0A3EDF0AD
:103D8D00D250E4900320F0A374BBF0A37480F090A4
:103D9D0002F2EAF0A3EDF0EA4401A3F09002EDE0A7
:103DAD00D394005003023F3943E6C043D10143C8C9
:103DBD000175C8607F08127B94400C7F10127B94B4
:103DCD004005C250023F168A8D75C8407F18127B80
:103DDD00944005C250023F16EBB401159002EAE083
:103DED00F58D75C8407F28127B944005C250023F67
:103DFD00169002EAE0A3E0F58D75C8407F28127B8E
:103E0D00944005C250023F1675C8607F08127B941E
:103E1D00400C7F10127B944005C250023F16EA44BD
:103E2D0001F58D75C8407F40127B944005C250024C
:103E3D003F16E49002F1F09002EDE0FF9002F1E008
:103E4D00FEC39F50579002EEE07031EF14B5060A95
:103E5D0075C8407F58127B94800875C8447F5012F6
:103E6D007B949002EFE0FEA3E0F5828E83E58DF06A
:103E7D009002EFE475F001122248801875C8447F56
:103E8D0050127B949002F1E024F5F582E43402F5B2
:103E9D0083E58DF09002F1E004F0809B9002EEE05E
:103EAD006401706575C8407F58127B94900320E5BE
:103EBD008DF07B017A0279F29002EDE02403FD1280
:103ECD007D46900320E0B5073EE49002F1F09002AC
:103EDD00EDE0FF9002F1E0FEC39F502D74F52EF53D
:103EED0082E43402F583E0FF9002EFE0FCA3E0F5FD
:103EFD00828C83EFF09002EFE475F001122248906E
:103F0D0002F1E004F080C7C25075C850E5C830E436
:103F1D001B53B1F8900321E07002A3E0600E9003F3
:0E3F2D002174FFF5F012224880E280E0A250DD
:013F3B002263
:107DAB0075C632E4F5E6F5D1758A2075D10275C832
:077DBB00407589FFF58D22E0
:0369800075C432A9
:10698300E4F5877598509002B7747FF0A374CCF048
:106993009002B7E0F59D759CCCE0FEA3E0FFFBE41D
:1069A300C39BFF74809EFEE49400FDE49400FCE42A
:1069B3007B10FAF9F8122279EC121F18A804A90522
:1069C300AA06AB077F557E557D507C44121C7D1271
:0D69D3001F568F9E439D80759A0A759BFF8D
:0169E0002294
:03102300027CB29A
:067CB200C0E0C083C082A7
:107CB800C086758600309808C2989002B6E599F09B
:027CC800D08664
:077CCA00D082D083D0E0322C
:104A890080B678FA71C46B0C64C760C25B2755EBBA
:104A990051074C7449A2458441AA3E0D3AAB384AA4
:104AA900354132682FBB2D382B7A29362715251425
:104AB900233121C320101E761CF41B881A79192F63
:104AC90017F816D215BC14DD13E212F41213113EB5
:104AD90010970FD50F1E0E700DCC0D3E0CA90C1B97
:104AE9000B940B140AA80A3309C5095B08F7089D3A
:104AF900084207EB0798074A070406BC06770636FB
:104B090005F705BD0584054D051904E804B9048BAD
:104B190004600436040E03E803C303A0037E035EA6
:104B2900033F0321030402E902CF02B6029E028673
:104B39000270025B02470232021F020D01FC01EB07
:104B490001DA01CB01BC01AE01A001920185017915
:104B5900016D01620156014B01410137012E01240A
:104B6900011B0113010B010300FB00F300EC00E53D
:104B790000DF00D800D200CC00C600C000BA00B5E2
:104B890000B000AB00A700A2009D0099009500911C
:104B9900008D008900850082007F007B0078007508
:104BA9000072006F006C0069006600640061005FBC
:104BB900005C005A0058005600530051004F004E47
:024BC900004C9E
:03100000027C73FC
:107C730075819F007808760008B8A0FAE4900000A8
:107C8300F0A3A882A983B8DCF7B907F4000230A6F1
:1039FC00A2AF924DC2AF900234E0FFA3E09003253A
:103A0C00CFF0A3EFF090022C12241E90034312244B
:103A1C008490023012241E90037612248490023675
:103A2C00E0FFA3E0900364CFF0A3EFF0900220122C
:103A3C00241E90037B122484900224E0FFA3E090C8
:103A4C000374CFF0A3EFF090021EE0FEA3E0FFE4BE
:103A5C00FCFD90034D12248485111C85121D850FCD
:103A6C001A85101B90035F1224A900000000E4903B
:103A7C000372F0A3F0A24D92AF90034C741EF09021
:103A8C00036B745AF0A3740BF0A3740FF0900366DD
:103A9C001224A9FFFF7748E490036AF090036F04A7
:103AAC00F09003877414F090033C743EF0A3748080
:103ABC00F0A3E4F0A37411F09003707406F0A374F7
:103ACC0022F0900389743CF0900003E02438FE90BF
:103ADC000002E034FF900323F0A3CEF09003577460
:103AEC000FF090035E740AF0900014E0FFA3E090D6
:103AFC00037FCFF0A3EFF090034B745AF0E513FB68
:103B0C007A007C117D94FF7E001221E1E4FCFD9093
:103B1C00032D1224847C0B7DB8AF037E001221E1AF
:103B2C00E4FCFD900353122484900363743CF090E6
:103B3C0003887414F0900331740FF090037A7414AA
:103B4C00F090036E740AF09003271224A900000071
:103B5C0028900342741EF0900340740BF0A3744140
:103B6C00F0900351740BF0A37441F0900381E4F0D6
:103B7C00A37432F0900347E4F0A37405F09003387B
:103B8C00E4F0A37469F0900383E4F0A37464F09000
:103B9C000349E4F0A3741EF090033AE4F0A37462BA
:103BAC00F09003857401F0A37490F090035CE4F042
:043BBC00A3744BF0B3
:013BC00022E2
:106E7800A2AF924DC2AF900325E0FFA3E090023489
:106E8800CFF0A3EFF090034312241E90022C12249B
:106E98008490037612241E90023012248490036496
:106EA800E0FFA3E0900236CFF0A3EFF0A25A9222BF
:106EB800A25B92209000B9E024FF9221A24D92AFEC
:016EC80022A7
:067F81005AA569963CC3FD
:104D03007F647E00E49002B9F09002B9E0FDC394A1
:104D13000A4003024E21ED25E02402F582E434002B
:104D2300F583E0FCA3E0D3951DEC951C5003024EE4
:104D3300189002B9E0705790007AE0FCA3E0FDD32D
:104D4300951DEC951C5003301906E4FEFF024E211D
:104D5300C3E51D9DFFE51C9CFE7C007D0A12252CEE
:104D6300EEC0E0EFC0E090007AE0FEA3E0FFC39066
:104D73000003E09FFF900002E09EFECBEFCBFAE43E
:104D8300F9F8D0E0FFD0E0FE122304024E21900296
:104D9300B9E025E02400F582E43400F583E0FEA3C6
:104DA300E0FFC3E51D9FFFE51C9EFE7C007D0A120C
:104DB300252CECC0E0EDC0E0EEC0E0EFC0E09002D7
:104DC300B9E0FF25E02400F582E43400F583E0FC3C
:104DD300A3E0FDEF25E02402F582E43400F583E04F
:104DE300FEA3E0C39DFFEE9CFECBEFCBFAE4F9F804
:104DF300D0E0FFD0E0FED0E0FDD0E0FC122304CDF4
:104E0300EFCDCCEECC9002B9E075F00AA42DFFE50E
:0F4E1300F03CFE80099002B9E004F0024D0C2241
:104270009002B9EEF0A3EFF09000AAE0F9FDD3EFC1
:104280009DEE9400500302434990036BE0FF9002BF
:10429000B9E0FCA3E0FDD39FEC94004078ED94647A
:1042A000EC940050709002B9E0FAA3E0FBC3746490
:1042B0009BFFE49AFE7C007D0A1221E1E9FDC3EB3D
:1042C0009DFDEA9CFCD3ED9FEC9E50030243DE90E3
:1042D00002B9E0FEA3E0FF9000AAF07C007D0A1284
:1042E00021E19003A8EEF0A3EFF09002B9E0FEA365
:1042F000E0FFE4FD90001AE0F8A3E0F9A3E0FAA3E0
:10430000E0FB122279E47B64FAF9F81223049000AE
:10431000AB122484229002B9E07004A3E0646460CC
:10432000030243DE9000AA7464F09003A87403F0C3
:10433000A374E8F090001AE0FCA3E0FDA3E0FEA364
:10434000E0FF9000AB122484229000AAE0FD9002CE
:10435000B9E0FEA3E0FFC3ED9FFDE49EFC90034C9B
:10436000E0FBD3ED9BEC9400403F9000AAEFF07C83
:10437000007D0A1221E19003A8EEF0A3EFF0900275
:10438000B9E0FEA3E0FFE4FD90001AE0F8A3E0F935
:10439000A3E0FAA3E0FB122279E47B64FAF9F812B5
:1043A00023049000AB122484229002B9E07002A38F
:1043B000E0702B9000AA04F09003A8E4F0A3740A24
:1043C000F0E47B64FAF9F890001AE0FCA3E0FDA3A6
:0F43D000E0FEA3E0FF1223049000AB122484222E
:1043DF001239FC124D039002B7EEF0A3EFF0E47F19
:1043EF00E87E03FDFC9000ABE0F8A3E0F9A3E0FA50
:1043FF00A3E0FB12227990001AE0F8A3E0F9A3E002
:10440F00FAA3E0FB1223049003A8EEF0A3EFF090C1
:10441F0002B7E0FEA3E0FF1242709000AAE0FF7E19
:10442F0000900325EEF0FAA3EFF0FB90001AE0FCEA
:10443F00A3E0FDA3E0FEA3E0FF900343122484CF8B
:10444F00EBCF7E00E4FCFD900343E0F8A3E0F9A37B
:10445F00E0FAA3E0FB122279E47B64FAF9F8122365
:10446F00049003761224849000ABE0FCA3E0FDA33C
:10447F00E0FEA3E0FF90035812248490033412242B
:10448F00A9000000009003A6E0FFA3E090032BCF4C
:10449F00F0A3EFF0E47830F608F67838F608F678FF
:1044AF0034122490000000009003AC1224A90000E5
:1044BF000000E490039CF0A3F09003B2F0A3F090FF
:1044CF0003AAF0A3F0C25BC257C2599003A5F090A4
:1044DF0003A4F0783AF608F67832F608F69003A8B7
:1044EF00E0FFA3E09003B0CFF0A3EFF0C25AC256A3
:1044FF009003B41224A900000000E49003A6F0A3D7
:10450F00F090038E1224A90000000090039712244C
:10451F00A9000000009003921224A900000000E4FB
:10452F0090039BF0900396F0C25890038A1224A92F
:08453F0000000000126E78225A
:10500000124D039002B7EEF0A3EFF0900331E0FFF2
:10501000E4FCFDFE90001AE0F8A3E0F9A3E0FAA397
:10502000E0FB122279E47B0AFAF9F8122304C8ECB7
:10503000C8C9EDC9CAEECACBEFCB90037BE0FCA395
:10504000E0FDA3E0FEA3E0FFD31223C7500302500C
:10505000D690037AE0FF7E009002B7E0FCA3E0FD6B
:10506000D39FEC9E4070D3900380E0951D90037F0A
:10507000E0951C4061ED9FFBEC9EFA9003A8E0FEDA
:10508000A3E0FF7C007D0A1221F3C3EF9BEE9A5050
:105090004590036EE0FFC39002B8E09FFF9002B717
:1050A000E09400FE7C007D0A1221E19003A8EEF05E
:1050B000A3EFF0E4FD90001AE0F8A3E0F9A3E0FA12
:1050C000A3E0FB122279E47BE87A03F9F8122304C7
:0750D0009000AB12248422C2
:102559001239FC900340E0FEA3E0FFD3900375E03D
:102569009F900374E09E401EE4FFFEFDFC900397DC
:10257900E0F8A3E0F9A3E0FAA3E0FBD31223B1400A
:1025890005301802D25BC3900380E0951D90037F4C
:10259900E0951C5012900396E004F0E09405400E7B
:1025A9007405F0D2578007C257E4900396F0900063
:1025B90028E0FEA3E0FFEE3395E0FDFC90037BE00D
:1025C900F8A3E0F9A3E0FAA3E0FBD31223B1500387
:1025D9000227C1E49003B2F0A3F09003AAF0A3F09C
:1025E90090039BE004F0E0D3940540057405F0D214
:1025F900589000B9E06010D25AE4F09003B4122464
:10260900A900000000C256900372E0FEA3E0FFEEAD
:102619003395E0FDFC900281E0F8A3E0F9A3E0FA2C
:10262900A3E02FFFEA3EFEE93DFDE83CFC90038E66
:10263900122484E4FFFEFDFC90038EE0F8A3E0F988
:10264900A3E0FAA3E0FBD31223B14021900281E079
:10265900A3E0A3E0FEA3E0FF900373E02FFF900344
:1026690072E03EFE783BEF26F618EE36F6C3783B6D
:10267900E6941018E6940E500302270B0874F0260E
:10268900F61874F136F690001AE0FCA3E0FDA3E019
:10269900FEA3E0FF9000ABE0F8A3E0F9A3E0FAA302
:1026A900E0FBC31223C750219000ABE0FCA3E0FD7F
:1026B900A3E0FEA3E02401FFE43EFEE43DFDE43C8B
:1026C900FC9000AB122484801490001AE0FCA3E073
:1026D900FDA3E0FEA3E0FF9000AB122484305A8DE5
:1026E9009003B4E0FCA3E0FDA3E0FEA3E02401FF16
:1026F900E43EFEE43DFDE43CFC9003B41224840274
:102709002676900340E0FEA3E0FFD3900375E09F97
:10271900900374E09E404490006AE0FEA3E0FFEE5F
:102729003395E0FDFC900281E0F8A3E0F9A3E0FA1B
:10273900A3E0FBC31223B15022C3900069E0951DA9
:10274900900068E0951C501390006CE0FF9003A581
:10275900E004F0C39F4004EFF0D25B90006AE0FE12
:10276900A3E0FFEE3395E0FDFC900281E0F8A3E0E1
:10277900F9A3E0FAA3E0FBC31223B1503590034D4E
:10278900E0FCA3E0FDA3E0FEA3E0FF90032DE0F849
:10279900A3E0F9A3E0FAA3E0FBC31223C750139007
:1027A9000363E0FF9003A4E004F0C39F4004EFF04B
:1027B900D259125000022AFF900028E0FEA3E0FF40
:1027C900C3E49FFFE49EFE3395E0FDFC90037BE0AC
:1027D900F8A3E0F9A3E0FAA3E0FBC31223B1400395
:1027E9000229B6E49003A5F09003A4F0C259C25B94
:1027F9009003AAF0A3F09003B3F090039BF0C258A2
:1028090090035FE0FCA3E0FDA3E0FEA3E0FF9002DC
:1028190081E0F8A3E0F9A3E0FAA3E02FFBEA3EFA8E
:10282900E93DF9E83CF8900372E0FEA3E0FFEE33DE
:1028390095E0FDFCEB2FFFEA3EFEE93DFDE83CFC9F
:1028490090038E12248490038EE0FCA3E0FDA3E0A4
:10285900FEA3E0FFEC33500AC37833E69FF618E68F
:102869009EF6C37833E6941018E6940E50030229B5
:102879004BC37833E6941018E6940E40670874F059
:1028890026F61874F136F69000B3E0FCA3E0FDA338
:10289900E0FEA3E02401FFE43EFEE43DFDE43CFC50
:1028A9009000B3122484E47F01FEFDFC9000ABE0AC
:1028B900F8A3E0F9A3E0FAA3E0FBD31223C740B1E0
:1028C9009000ABE0FCA3E0FDA3E0FEA3E024FFFF42
:1028D900EE34FFFEED34FFFDEC34FFFC9000AB124B
:1028E9002484808D90001EE0FCA3E0FDA3E0FEA3FC
:1028F900E0FF9000B3E0F8A3E0F9A3E0FAA3E0FB5E
:10290900C31223C7403C9000B3E0FCA3E0FDA3E061
:10291900FEA3E0FF90001EE0F8A3E0F9A3E0FAA30C
:10292900E0FBEF9BFFEE9AFEED99FDEC98FC900021
:10293900B3122484900023E004F07006900022E092
:1029490004F0900351E0FEA3E0FFD3900375E09FEC
:10295900900374E09E5003022AFF9000AFE0FCA3AD
:10296900E0FDA3E0FEA3E0FF900281E0F8A3E0F917
:10297900A3E0FAA3E0FBD31223B15003022AFFD349
:1029890090007BE0951B90007AE0951A5003022A8B
:10299900FF90007CE0FF9003B2E004F09F50030237
:1029A9002AFFEFF09000B97401F0022AFF90037238
:1029B900E0FAA3E0FBFFCEEACEEE3395E0FDFC336F
:1029C9004003022AA9C37833E69BFF18E69AFEF66C
:1029D90008EFF6C39410EE940E5003022AA974F07E
:1029E90026F61874F136F69000B3E0FCA3E0FDA3D7
:1029F900E0FEA3E02401FFE43EFEE43DFDE43CFCEF
:102A09009000B3122484E47F01FEFDFC9000ABE04A
:102A1900F8A3E0F9A3E0FAA3E0FBD31223C740220D
:102A29009000ABE0FCA3E0FDA3E0FEA3E024FFFFE0
:102A3900EE34FFFEED34FFFDEC34FFFC9000AB12E9
:102A4900248490001EE0FCA3E0FDA3E0FEA3E0FFC8
:102A59009000B3E0F8A3E0F9A3E0FAA3E0FBC31206
:102A690023C7403C9000B3E0FCA3E0FDA3E0FEA334
:102A7900E0FF90001EE0F8A3E0F9A3E0FAA3E0FB71
:102A8900EF9BFFEE9AFEED99FDEC98FC9000B312D6
:102A99002484900023E004F07006900022E004F002
:102AA900900389E0FF9003AAE475F001122248FC23
:102AB900C3E5F09FEC9400403A900351E0FEA3E097
:102AC900FFD3900375E09F900374E09E4025D39057
:102AD900007BE0951B90007AE0951A401690007CE7
:102AE900E0FF9003B3E004F09F4008EFF09000B9D5
:102AF9007401F0123394E47FE87E03FDFC9000AB8F
:102B0900E0F8A3E0F9A3E0FAA3E0FB122279900030
:102B19001AE0F8A3E0F9A3E0FAA3E0FB122304907A
:102B290003A8EEF0A3EFF0900028E0FEA3E0FFC3B6
:102B3900E49FFFE49EFE3395E0FDFC90037BE0F803
:102B4900A3E0F9A3E0FAA3E0FBC31223B1400C20F0
:102B59001509201A06201B03301C02C25A121056EE
:102B69009000AAE0FF7E00900325EEF0FAA3EFF0B3
:102B7900FB90001AE0FCA3E0FDA3E0FEA3E0FF90B8
:102B89000343122484CFEBCF7E00E4FCFD90034382
:102B9900E0F8A3E0F9A3E0FAA3E0FB122279E47BD1
:102BA90064FAF9F81223049003761224849000221F
:102BB900E0FFA3E0900364CFF0A3EFF09003A8E057
:102BC900FFA3E09003B0CFF0A3EFF090038EE0FCF9
:102BD900A3E0FDA3E0FEA3E0FF90039712248490F5
:102BE90000ABE0FCA3E0FDA3E0FEA3E0FF900358E7
:102BF9001224849003ACE0FCA3E0FDA3E0FEA3E073
:102C0900FF9003341224849003A6E0FFA3E090030D
:0A2C19002BCFF0A3EFF0126E78222B
:1079C3001239FC90038A122443900327E0F8A3E0C2
:1079D300F9A3E0FAA3E0FBC31223C75014900327D3
:1079E300E0FCA3E0FDA3E0FEA3E0FF90038A1224E2
:0579F30084126E7822F1
:1035EC009005FCE4F0A37464F01239FC124D0390C6
:1035FC0005FCEEF0A3EFF04E702E9000AA04F090B4
:10360C0003A8E4F0A3740AF0E47B64FAF9F89000E0
:10361C001AE0FCA3E0FDA3E0FEA3E0FF122304905C
:10362C0000AB1224840236F6900327E0FCA3E0FDE5
:10363C00A3E0FEA3E0FF90038AE0F8A3E0F9A3E087
:10364C00FAA3E0FBC31223C7400E9005FCE0FEA3D7
:10365C00E0FF1242700236F6E47F64FEFDFC90003F
:10366C001AE0F8A3E0F9A3E0FAA3E0FB12227990A8
:10367C0000ABE0F8A3E0F9A3E0FAA3E0FB1223040B
:10368C00C8ECC8C9EDC9CAEECACBEFCB90034CE06D
:10369C00FF9005FDE02FFF9005FCE03400FEE4FCFC
:1036AC00FDD31223C740439005FCE0FAA3E0FB7C5A
:1036BC00007D0AFFCEEACE1221E19003A8EEF0A322
:1036CC00EFF0CFEBCFCEEACEE4FD90001AE0F8A3FA
:1036DC00E0F9A3E0FAA3E0FB122279E47B64FAF9A7
:1036EC00F81223049000AB122484E47830F608F628
:1036FC007838F608F6783412249000000000900315
:10370C00AC1224A900000000E490039CF0A3F090FC
:10371C0003B2F0A3F09003AAF0A3F0C25BC257C2AD
:10372C00599003A5F09003A4F0783AF608F6783295
:10373C00F608F69003A8E0FFA3E09003B0CFF0A347
:10374C00EFF0C25AC2569003B41224A90000000034
:10375C00E49003A6F0A3F090038E1224A9000000BD
:10376C00009003971224A9000000009003921224E9
:10377C00A900000000E490039BF0900396F0C2585F
:10378C0090038A1224A9000000009000AAE0FF7E9A
:10379C0000900325EEF0FAA3EFF0FB90001AE0FC8A
:1037AC00A3E0FDA3E0FEA3E0FF900343122484CF2B
:1037BC00EBCF7E00E4FCFD900343E0F8A3E0F9A31B
:1037CC00E0FAA3E0FB122279E47B64FAF9F8122305
:1037DC00049003761224849000ABE0FCA3E0FDA3DC
:1037EC00E0FEA3E0FF9003581224849003341224CB
:1037FC00A900000000E490032BF0A3F0126E7822D5
:10339400305A09305B06C25AD2568021305B1E90E7
:1033A40003A87403F0A374E8F090001AE0FCA3E00F
:1033B400FDA3E0FEA3E0FF9000AB1224843056038B
:1033C4000234449000B7E0FCA3E0FD900022E0FE4C
:1033D400A3E0FFC39DFDEE9CFCC390035DE09D90C4
:1033E400035CE09C40030235EB205B030235EB12E7
:1033F4006AFEE4FCFDFE90001AE0F8A3E0F9A3E005
:10340400FAA3E0FB122279ECC0E0EDC0E0EEC0E0EC
:10341400EFC0E09000B7E0FEA3E0FF126AFECBEF3E
:10342400CBE4FAF9F8D0E0FFD0E0FED0E0FDD0E044
:10343400FC1223049003B41224840235A00235A0A4
:10344400C256E47F32FEFDFC900016E0F8A3E0F9DA
:10345400A3E0FAA3E0FB122279E47B64FAF9F81200
:1034640023049002B71224849002B7E0FCA3E0FD89
:10347400A3E0FEA3E0FF9003B4E0F8A3E0F9A3E027
:10348400FAA3E02FFFEA3EFEE93DFDE83CFC900094
:1034940016E0F8A3E0F9A3E0FAA3E0FBC31223C704
:1034A40040030235EB900342E0FFE4FCFDFE900094
:1034B4001AE0F8A3E0F9A3E0FAA3E0FB122279E40E
:1034C4007B64FAF9F81223049002B7122484900260
:1034D400B7E0FCA3E0FDA3E0FEA3E0FF90001AE048
:1034E400F8A3E0F9A3E0FAA3E02FFFEA3EFEE93DEA
:1034F400FDE83CFC9003B4E0F8A3E0F9A3E0FAA3F0
:10350400E0FBD31223C7402E9002B7E0FCA3E0FDFA
:10351400A3E0FEA3E0FF90001AE0F8A3E0F9A3E023
:10352400FAA3E02FFFEA3EFEE93DFDE83CFC9003F0
:10353400B412248480669002B7E0FCA3E0FDA3E00B
:10354400FEA3E0FF9003B4E0F8A3E0F9A3E0FAA33C
:10355400E02FFFEA3EFEE93DFDE83CFC90001AE066
:10356400F8A3E0F9A3E0FAA3E0FBD31223C7402CAD
:103574009002B7E0F8A3E0F9A3E0FAA3E0FB90001F
:103584001AE0FCA3E0FDA3E0FEA3E09BFFEE9AFE9D
:10359400ED99FDEC98FC9003B41224849003B4E0FC
:1035A400FCA3E0FDA3E0FEA3E0FF90001A12248434
:1035B4009003A87403F0A374E8F090001AE0FCA34D
:1035C400E0FDA3E0FEA3E0FF9000AB122484900092
:1035D40022E0FFA3E09000B7CFF0A3EFF09003B494
:0835E4001224A90000000022DE
:106AFE00C3900386E09F900385E09E5004795580F5
:106B0E0048C3900384E09F900383E09E5016900349
:106B1E0049E0FCA3E0FD1221F390033AE0A3E0C3A9
:106B2E009FF98025C3900382E09F900381E09E50E1
:106B3E0016900347E0FCA3E0FD1221F3900338E02A
:0D6B4E00A3E0C39FF980027964CFE9CF2254
:10105600E49002B7F0A3F0FFA3F0A3F0A3F090038F
:101066009EE0645A6028A2AF924DC2AF75A701E414
:10107600EF90124093FE749E2FF582E43403F583BD
:10108600EEF00FEFB406E9E4F5A7A24D92AF900398
:10109600A3E064C36003021C48FF749E2FF582E43C
:1010A6003403F583E0FEEF907F81936E6003021CAC
:1010B600480FEFB406E48003021C48900028E0FEC7
:1010C600A3E0FFEE3395E0FDFC90037BE0F8A3E0A0
:1010D600F9A3E0FAA3E0FBD31223B150030214F103
:1010E6002058030214F1E47830F608F67838F6084A
:1010F600F69000AAE0D394634003021C48C3900311
:1011060080E0951D90037FE0951C401E90034BE008
:10111600FF7E007C007D0A1221E1D39003A9E09FA7
:101126009003A8E09E50030213C930575A90034B10
:10113600E0FBFF7E007C007D0A1221E19003A9E01E
:101146002496FD9003A8E03400FCC3ED9FEC9E506E
:1011560036EBFF7E007C007D0A1221E1EEF0A3EF64
:10116600F0CFEBCFE4FDFE90001AE0F8A3E0F9A380
:10117600E0FAA3E0FB122279E47B64FAF9F8122381
:10118600049000AB12248490034DE0FCA3E0FDA381
:10119600E0FEA3E0FF90032DE0F8A3E0F9A3E0FA58
:1011A600A3E0FBD31223C7500302123090034DE095
:1011B600F8A3E0F9A3E0FAA3E0FB90032DE0FCA37B
:1011C600E0FDA3E0FEA3E09BFBEE9AFAED99F9ECB5
:1011D60098F8900387E0FFE4FCFDFE122279E47B99
:1011E6000AFAF9F8122279EEC0E0EFC0E090001496
:1011F600E0FEA3E0FFC3900069E09FFF900068E077
:101206009EFECBEFCBFAE4F9F8D0E0FFD0E0FE1279
:101216002304EFC0E0AF13CBEFCBE4FAF9F8D0E04C
:10122600FF122304900392122484C3900063E09576
:101236001DFF900062E0951CFE900387E0FD7C0098
:1012460012252CE47B0AFAF9F8122279EEC0E0EFB7
:10125600C0E0900014E0FEA3E0FFC3900069E09FA9
:10126600FF900068E09EFECBEFCBFAE4F9F8D0E001
:10127600FFD0E0FE1223049002BC12248490039255
:10128600E0FCA3E0FDA3E0FEA3E0FF9002BCE0F8D3
:10129600A3E0F9A3E0FAA3E0FBC31223C75014901E
:1012A60002BCE0FCA3E0FDA3E0FEA3E0FF900392F6
:1012B600122484E47F24FEFDFC90001AE0F8A3E0EB
:1012C600F9A3E0FAA3E0FB122279900392E0F8A3D7
:1012D600E0F9A3E0FAA3E0FB122279EEC0E0EFC04A
:1012E600E09000AAE0FFC374659FFFE49400FECB84
:1012F600EFCBFAE4F9F8D0E0FFD0E0FE122304E4E5
:101306007B0AFAF9F81223049003921224849000BF
:101316006AE0FEA3E0FFEE3395E0FDFC90038EE06D
:10132600F8A3E0F9A3E0FAA3E0FBD31223B1406CE3
:1013360090038EE0FCA3E0FDA3E0FEA3E0FFC8EC73
:10134600C8A3E0FCA3E0FDA3E0FEA3E0FF12230494
:10135600ECC0E0EDC0E0EEC0E0EFC0E090006AE077
:10136600FEA3E0FFFBCAEECAEA3395E0F9F8900364
:101376008EE0FCA3E0FDA3E0FEA3E0C39BFFEE9A94
:10138600FEED99FDEC98FCD0E0FBD0E0FAD0E0F958
:10139600D0E0F8122279900392122484900063E040
:1013A60024FFFF900062E034FFFEC3E51D9FE51CAD
:1013B6009E50030214839003921224A90000000099
:1013C6000214839003A8E0FEA3E0FF7C007D0A12CE
:1013D60021F3EF2401FFE43EFE9000AAE0FB7A0031
:1013E600C39FEA9E503C9003A8E0FEA3E0FF7C006A
:1013F6007D0A1221F3EB2401FDEA33FCD3ED9FECC9
:101406009E401FE47F24FEFDFC90001AE0F8A3E056
:10141600F9A3E0FAA3E0FB12227990039212248446
:10142600805B9000ABE0F8A3E0F9A3E0FAA3E0FB51
:1014360090001AE0FCA3E0FDA3E0FEA3E0C39BFF3F
:10144600EE9AFEED99FDEC98FCE47B107A0EF9F825
:10145600122279EEC0E0EFC0E09000AAE0FFC3746C
:10146600649FFFE49400FECBEFCBFAE4F9F8D0E0FA
:10147600FFD0E0FE12230490039212248490038E80
:10148600E0FCA3E0FDA3E0FEA3E0FFFBCAEECAC9B1
:10149600EDC9C8ECC8A3E0FCA3E0FDA3E0FEA3E011
:1014A600FF1223049002BAEEF0A3EFF020590330A6
:1014B6005B0D900388E0FF9002BAE4F0A3EFF09092
:1014C60003A6E475F001122248FEC39002BBE09524
:1014D600F09002BAE09E4003021C489000AAE00485
:1014E600F0E49003A6F0A3F0021C48900028E0FE6A
:1014F600A3E0FFC3E49FFFE49EFE3395E0FDFC906E
:10150600037BE0F8A3E0F9A3E0FAA3E0FBC3122310
:10151600B14003021BE89000AAE094015003021CAC
:1015260048900323E0FEA3E0FFAD137C0012252CB8
:1015360090034DE0F8A3E0F9A3E0FAA3E0FBC312A1
:1015460023C7402DD390007BE0951B90007AE09551
:101556001A501E900357E0FF7E007C007D0A122180
:10156600E1C39003A9E09F9003A8E09E4003021800
:101576000B90036CE0FEA3E0FFD3900375E09F9011
:101586000374E09E500302180B900366E0FCA3E090
:10159600FDA3E0FEA3E0FF90037BE0F8A3E0F9A340
:1015A600E0FAA3E0FBD31223B1500302180B7839FB
:1015B600E61846700302180B900397E0FCA3E0FDC3
:1015C600A3E0FEA3E024D0FFEE3407FEE43DFDE4F5
:1015D6003CFC90038EE0F8A3E0F9A3E0FAA3E0FB5D
:1015E600C31223B1400302180B900397E0FCA3E05B
:1015F600FDA3E0FEA3E02430FFEE34F8FEED34FF59
:10160600FDEC34FFFC90038EE0F8A3E0A3E0A3E03A
:10161600D31223B1500302180B90035EE07E00251F
:101626001BFFEE351AFEC3EF783996EE1896400387
:101636000217FA90039CE0FEA3E0FF9400EE9400EC
:1016460050030217FAEF9401EE9400500890039CA1
:10165600E4F0A304F090034DE0FCA3E0FDA3E0FE5C
:10166600A3E0FF783412242AD31223C750030217AB
:1016760013900353E0F8A3E0F9A3E0FAA3E0FB908C
:10168600034DE0FCA3E0FDA3E0FEA3E09BFBEE9A86
:10169600FAED99F9EC98F890039CE0FEA3E0FFE4DC
:1016A600FCFD122279ECC0E0EDC0E0EEC0E0EFC038
:1016B600E090034DE0F8A3E0F9A3E0FAA3E0FBE82D
:1016C600C0E07834122412D0E0F8C3EF9BFBEE9A08
:1016D600FAED99F9EC98F8D0E0FFD0E0FED0E0FD05
:1016E600D0E0FC122304EEC0E0EFC0E09000AAE0D8
:1016F60024FFFFE434FFFECBEFCBFAE4F9F8D0E0A9
:10170600FFD0E0FE1223049003921224849000740A
:10171600E0FEA3E0FFC3E51B9FFFE51A9EFE9003D4
:101726009CE0FCA3E0FD12252CEEC0E0EFC0E0C378
:101736007839E6951BFF18E6951AFECBEFCBFAE44F
:10174600F9F8D0E0FFD0E0FE122304EEC0E0EFC0CF
:10175600E09000AAE024FFFFE434FFFECBEFCBFAD3
:10176600E4F9F8D0E0FFD0E0FE1223049002BC12A8
:101776002484900392E0FCA3E0FDA3E0FEA3E0FF37
:101786009002BCE0F8A3E0F9A3E0FAA3E0FBC312E1
:1017960023C750149002BCE0FCA3E0FDA3E0FEA327
:1017A600E0FF9003921224847838A61A08A61B90AC
:1017B600034DE0FCA3E0FDA3E0FEA3E0FF783412B6
:1017C6002478E490039CF0A3F0900392E0F8A3E061
:1017D600F9A3E0FAA3E0FB90038EE0FCA3E0FDA3EF
:1017E600E0FEA3E0FF1223A31222799003921224B3
:1017F60084021B7690039DE004F0700690039CE043
:1018060004F0021B767838A61A08A61B90034DE052
:10181600FCA3E0FDA3E0FEA3E0FF7834122478E405
:1018260090039CF0A3F090036CE0FEA3E0FFC3904E
:101836000375E09F900374E09E4021900366E0FCF0
:10184600A3E0FDA3E0FEA3E0FF90037BE0F8A3E0A6
:10185600F9A3E0FAA3E0FB1223B1501D90001AE0B1
:10186600FCA3E0FDA3E0FEA3E0FF9003AC122484FA
:10187600E47830F608F60219FA7830E6FE08E6FF54
:101886002414FDE43EFC900374E0FAA3E0FBD39D30
:10189600EA9C5011EB2414FDE43AFCD3EF9DEE9C38
:1018A60050030219FA900374E0FEA3E0FF7830EECD
:1018B600F608EFF62487FFEE34F59002B7F0A3EFB3
:1018C600F090033EE0FEA3E0FFFBCAEECAE4F9F89F
:1018D6009002B7E0FEA3E0FFEE3395E0FDFC122296
:1018E60079C8ECC8C9EDC9CAEECACBEFCB90033CA8
:1018F600E0FEA3E0FFE4C3EF9BFBEE9AFAE499F95E
:10190600E498F89002B7E0FEA3E0FFEE3395E0FD21
:10191600FC122279E47B107A27F9F8127602C8ECD9
:10192600C8C9EDC9CAEECACBEFCB900370E0FEA3DF
:10193600E0FFE4FCFDEB2FFFEA3EFEED39FDEC385F
:10194600FC90001AE0F8A3E0F9A3E0FAA3E0FB128A
:101956002279E47BD07A07F9F81223049003AC12BB
:10196600248490001AE0FCA3E0FDA3E0FEA3E0FFC0
:101976009003ACE0F8A3E0F9A3E0FAA3E0FBD312EE
:1019860023C7401690001AE0FCA3E0FDA3E0FEA3E7
:10199600E0FF9003AC122484805AE47F06FEFDFC2F
:1019A60090001AE0F8A3E0F9A3E0FAA3E0FB122204
:1019B60079E47B0AFAF9F81223049003ACE0F8A361
:1019C600E0F9A3E0FAA3E0FBC31223C75026E47FA5
:1019D60006FEFDFC90001AE0F8A3E0F9A3E0FAA3E6
:1019E600E0FB122279E47B0AFAF9F8122304900349
:1019F600AC1224849003ACE0F8A3E0F9A3E0FAA3C8
:101A0600E0FB90001AE0FCA3E0FDA3E0FEA3E0C328
:101A16009BFFEE9AFEED99FDEC98FCE47B0DFAF93E
:101A2600F8122279E47B0AFAF9F81223049000AB43
:101A3600E0F8A3E0F9A3E0FAA3E0FBC31223C75042
:101A460020E47F24FEFDFC90001AE0F8A3E0F9A351
:101A5600E0FAA3E0FB122279900392122484021B7F
:101A6600769000ABE0FCA3E0FDA3E0FEA3E0FF90D0
:101A760003ACE0F8A3E0F9A3E0FAA3E02FFFEA3E07
:101A8600FEE93DFDE83CFC90001AE0F8A3E0F9A36E
:101A9600E0FAA3E0FBC3EF9BFFEE9AFEED99FDECA7
:101AA60098FCE47B64FAF9F81222799003ACE0F82A
:101AB600A3E0F9A3E0FAA3E0FB1223049002B9EF36
:101AC600F02401FFE433FE9000AAE0FDC39FEE641C
:101AD60080F87480985035ED2401FFE433FE9002BF
:101AE600B9E0FDD3EF9D7480F86E98401FE47F2423
:101AF600FEFDFC9003ACE0F8A3E0F9A3E0FAA3E056
:101B0600FB12227990039212248480649000ABE049
:101B1600FCA3E0FDA3E0FEA3E0FF9003ACE0F8A386
:101B2600E0F9A3E0FAA3E02FFFEA3EFEE93DFDE877
:101B36003CFC90001AE0F8A3E0F9A3E0FAA3E0FB6E
:101B4600C3EF9BFFEE9AFEED99FDEC98FCE47B104B
:101B56007A0EF9F8122279EFC0E09000AAE0FFFBB6
:101B6600E4FAF9F8D0E0FF122304900392122484D9
:101B760090038EE0FCA3E0FDA3E0FEA3E0FF1223AA
:101B8600A3CBEFCBCAEECAC9EDC9C8ECC8A3E0FC2B
:101B9600A3E0FDA3E0FEA3E0FF1223049002BAEE49
:101BA600F0A3EFF09003A6E475F001122248FCD3EF
:101BB600E5F09FEC9E400D9000AAE014F0E490033F
:101BC600A6F0A3F030197B90036FE0FF9000AAE027
:101BD600D39F506E90036AE060689000AA7401F08B
:101BE6008060E47838F608F6783412249000000015
:101BF60000E47830F608F69000AAE0D3940140425B
:101C0600900372E0FEA3E0FFEE3395E0FDFC335057
:101C1600319003A8E0FEA3E0FF7C007D0A1221F3C9
:101C2600CAEECACBEFCB9003B0E0FEA3E0FF7C0088
:101C36007D0A1221F3D3EF9BEE9A40069000AAE0AC
:101C460014F0E4FFFEFDFC900397E0F8A3E0F9A38F
:101C5600E0FAA3E0FBD31223B14009301806900046
:101C6600AA7464F09002BAE0FFA3E0900332CFF0CA
:041C7600A3EFF022C6
:107D2900304C19204306204403304510C24CC2434D
:0D7D3900C244C245C2AF127E861200A622CF
:10000000020D7A021003000000000002100B000035
:10001000000000021013000000000002101B00008E
:10002000000000021023000000000002102B00005E
:10003000000000021033000000000002103B00002E
:10004000000000021043000000000002104B0000FE
:10005000000000021053000000000002105B0000CE
:10006000000000021063000000000002106B00009E
:10007000000000021073000000000002107B00006E
:10008000000000021083000000000002108B00003E
:10009000000000021093000000000002109B00000E
:1000A0000000000210A3E4F526F525F524F523F55C
:1000B00030F52FF52EF52DF52C120D5E209803024C
:1000C000018E7400252BF582E43402F583E599F066
:1000D000052BE52BC3948C4003E4F52BE52BB401F1
:1000E0000D900200E0645A700302018C806BE52BD6
:1000F000B40214900201E064A56002805CE4F53172
:10010000F532F52202018C900202E0FF7E00240904
:10011000FDEE33FCAB2B7A00C3EB9DEC6480F874EE
:1001200080985062EF2407FFEE33FED3EB9FEE641E
:1001300080F8748098501574FF252BF582E4340103
:10014000F583E02532F532E43531F531E52BB405A0
:100150000D900204E064076033E4F52B802EE52B5C
:1001600064067028900205E0FF6406601FEF6407D4
:10017000601AEF64086015EF64096010EF640A60AC
:100180000B432230800653B1F8120A9DC298309971
:100190004453B1F8900202E02408FFE433FEC3E5C3
:1001A0002B9FEE6480F87480984013E4F586D29C0F
:1001B000F52B900200F0A3F0A3F0D2028015052BDE
:1001C000E4F586C29C7400252BF582E43402F583A5
:1001D000E0F599C299E52C640A60030200BC53B1B2
:1001E000F82002030200BCC202F52C12000002003B
:1001F000BCC200900206E0FFC395214014E5212413
:1002000004FDE433FCD3EF9DEC6480F874809840E7
:100210000A900206E060047405F022900206E0F500
:1002200021E4F0900202E070152526F526E525343C
:1002300002F525E43524F524E43523F52322E521D0
:100240005403F50AE4F508F509900202E0FD7C008C
:10025000C3E5099DE5089C503274072509F582E441
:100260003402F583E0FBAF0A7E00120638E5092F61
:10027000FFE5083EFE74002FF58274003EF583EB27
:10028000F00509E50970C2050880BEE50A6403604F
:100290000302044F751D551208955003020386E4AE
:1002A000FF7E02FDFCAB26AA25A924A8231207186D
:1002B000401AE5269400F526E5259402F525E52467
:1002C0009400F524E5239400F5238009E4F526F550
:1002D00025F524F523E4F50F30015E2526F50EE51E
:1002E000253410F50DE43524F50CE43523F50BE445
:1002F000252AFFE529340CFEE43528FDE43527FCEA
:10030000AB0EAA0DA90CA80BC31207184040E42598
:100310002AFBE529340CFAE43528F9E43527F8C33B
:10032000E50E9BF50EE50D9AF50DE50C99F50CE53E
:100330000B98F50B750F018015E42526F50EE525C4
:100340003484F50DE43524F50CE43523F50B751DE7
:1003500055AF0EAE0DAD0CAC0B850F15120B7EAF6D
:100360000EAE0DAD0CAC0B850F15120C8C500E1291
:10037000089540129002067403F002044C900206A5
:100380007402F002044CE4F50A75F004E50AA424B2
:1003900002F582E5F03400F583E0FFE4FCFDFE7831
:1003A0001012073CC004C005C006C00775F004E584
:1003B0000AA42403F582E5F03400F583E0FFE4FCB1
:1003C000FDFE781812073CD003D002D001D000EF18
:1003D0004BFFEE4AFEED49FDEC48FCC004C005C0F1
:1003E00006C00775F004E50AA42401F582E5F0349F
:1003F00000F583E0FFE4FCFDFE780812073CD00323
:10040000D002D001D000EF4BFBEE4AFAED49F9ECF7
:1004100048F875F004E50AA42400F582E5F03400FC
:10042000F583E0FFEB4FFFEAFEE9FDE8FCE5302F46
:10043000F530E52F3EF52FE52E3DF52EE52D3CF56B
:100440002D050AE50A64806003020389E4F51D2294
:10045000E4F526F525F524F523F530F52FF52EF5F1
:100460002DF52AF529F528F527900209E0FFE4FC8F
:10047000FDFE781012073CC004C005C006C007A3EB
:10048000E0FFE4FCFDFE781812073CD003D002D058
:1004900001D000EF4BFFEE4AFEED49FDEC48FCC0F9
:1004A00004C005C006C007900208E0FFE4FCFDFEA2
:1004B000780812073CD003D002D001D000EF4BFBEC
:1004C000EE4AFAED49F9EC48F8900207E0FFEB4FED
:1004D000F52AEAF529E9F528E8F527200006900233
:1004E00006740AF0E4FF7E78FDFCAB2AAA29A9284D
:1004F000A827D312071840052001028017E4FF7EC9
:10050000ECFDFCAB2AAA29A928A827D3120718407A
:100510000A3001079002067401F022E4900206F00E
:10052000F521751D55F515FF7E0EFDFC120B7EE4C1
:10053000F515FF7E0EFDFC120C8C502B30012E7534
:100540001BA5E4F51C7FFF7E0FFDFC120B15E4F5E7
:100550001B7FFF7E0FFDFC120D94EF64A5600E90D3
:1005600002067403F080069002067402F0E4F51DA2
:10057000900206E06003020631FB7A02F9F8AF2A26
:10058000AE29AD28AC271206868F09E4F508E508E8
:10059000C395094003020637E4F50A300107F50E5A
:1005A000750D108006E4F50E750D84F50CF50BE560
:1005B0000825E0FEE4FCFD250EF50EE50D3EF50DEB
:1005C000ED350CF50CEC350BF50B300135E5092458
:1005D000FEFBE434FFFAED34FFF9EC34FFF8AF082A
:1005E000E4FED3120718501A750A01E5082402FF29
:1005F000C3EF9509FFEF25E0FEE4F50E8E0DF50C37
:10060000F50B751D55AF0EAE0DAD0CAC0B850A1577
:10061000120B7EAF0EAE0DAD0CAC0B850A15120C95
:100620008C40069002067402F0E4F51D05080205F0
:100630008E9002067405F022EF8DF0A4A8F0CF8C06
:10064000F0A428CE8DF0A42EFE2275F0087582004D
:10065000EF2FFFEE33FECD33CDCC33CCC58233C587
:10066000829BED9AEC99E58298400CF582EE9BFE18
:10067000ED9AFDEC99FC0FD5F0D6E4CEFBE4CDFA73
:10068000E4CCF9A88222B800C1B90059BA002DEC17
:100690008BF084CFCECDFCE5F0CBF97818EF2FFFAF
:1006A000EE33FEED33FDEC33FCEB33FB10D7039957
:1006B0004004EB99FB0FD8E5E4F9FA227818EF2F04
:1006C000FFEE33FEED33FDEC33FCC933C910D70523
:1006D0009BE99A4007EC9BFCE99AF90FD8E0E4C942
:1006E000FAE4CCFB2275F010EF2FFFEE33FEED3372
:1006F000FDCC33CCC833C810D7079BEC9AE899409F
:100700000AED9BFDEC9AFCE899F80FD5F0DAE4CD00
:10071000FBE4CCFAE4C8F922EB9FF5F0EA9E42F044
:10072000E99D42F0E89C45F022E8600FECC313FC21
:10073000ED13FDEE13FEEF13FFD8F122E8600FEF8B
:10074000C333FFEE33FEED33FDEC33FCD8F122EC86
:100750008EF0A4CCC5F0CCCDF8EFA4CEC5F02DFD25
:10076000E43CFCE8A42EC8C5F03DFDE43CFCEFA44D
:10077000FFE5F028FEE43DFDE43CFC22E4F50853EF
:10078000B1F8E508C3943A501FE4F50AAF08FE7CBF
:1007900002FD12074FE42FF510EE3410F50FE43D83
:1007A000F50EE43CF50D8021750A01AF087E007C52
:1007B000027D0012074FE42FF510EE348CF50FED9B
:1007C00034FFF50EEC34FFF50D751D55AF10AE0F6F
:1007D000AD0EAC0D850A15120B7EAF10AE0FAD0E2F
:1007E000AC0D850A15120C8C4003020883E4F50B4E
:1007F000F50CAE0BAF0CE4FCFDFB7A02F9F8D3125A
:1008000007185003020886AF087E007C027D0012A4
:10081000074FA804A905AA06AB07E4250CFFE50BC2
:100820003484FEE433FDE433FCEB2FFFEA3EFEE9C3
:100830003DFDE83CFCE4F51B120D948F09E50C2509
:1008400010FFE50B350FFEE4350EFDE4350DFC859C
:10085000091B850A1C120B15E50C2510FFE50B354D
:100860000FFEE4350EFDE4350DFC850A1B120D94D8
:10087000EF650960037F0222050CE50C7002050B91
:100880000207F27F01220508E508C3943C500302E9
:10089000077F7F0022D203E4F510F511AE10AF11EF
:1008A000E4FCFDFB7A02F9F8D312071850030209A1
:1008B0008CE4F51630015E2526F515E5253410F596
:1008C00014E43524F513E43523F512E4252AFFE575
:1008D00029340CFEE43528FDE43527FCAB15AA14B9
:1008E000A913A812C31207184040E4252AFBE529E2
:1008F000340CFAE43528F9E43527F8C3E5159BF5FF
:1009000015E5149AF514E51399F513E51298F51207
:100910007516018015E42526F515E5253484F514B2
:10092000E43524F513E43523F512AF15AE14AD13F9
:10093000AC1274002511F58274003510F583E0F5D2
:100940001B85161C120B15AF15AE14AD13AC12851A
:10095000161B120D9474002511F58274003510F5E4
:1009600083E06F6004C2038023E5262401F526E4BA
:100970003525F525E43524F524E43523F523051143
:10098000E511600302089C051002089CA203227E68
:10099000007D007C00900209E0FFE4781012073C23
:1009A000C004C005C006C007A3E0FFE4FCFDFE785C
:1009B0001812073CD003D002D001D000EF4BFFEE5D
:1009C0004AFEED49FDEC48FCC004C005C006C00766
:1009D000900208E0FFE4FCFDFE780812073CD0031B
:1009E000D002D001D000EF4BFBEE4AFAED49F9EC12
:1009F00048F8900207E0FFEB4FFFEAFEE9FDE8FC54
:100A0000AB30AA2FA92EA82DC31207186007900299
:100A1000067408F022E4900206F022E4F508F509D5
:100A2000900202F0900205740BF0900203E0FFA325
:100A3000E0900203F0A3EFF07F02900202E0FE24B8
:100A400007FDE433FCEFC39DEC6480F8748098509C
:100A50001774002FF582E43402F583E02509F509C7
:100A6000E43508F5080F80D274072EF582E43402CD
:100A7000F583E509F0E508FF900202E02408F5821D
:100A8000E43402F583EFF0C202E4F586C29C740000
:100A9000252BF582E43402F583E0F59922E4F52B69
:100AA000900202E0FD2408F582E43402F583E0FEC2
:100AB00074072DF582E43402F583E07C002400FF06
:100AC000EC3EFEEF65327003EE6531600343228039
:100AD000E5226006900206F08038900205E0FEB440
:100AE0000605120CD5802BEEB407051204508022A7
:100AF000900205E0B408051201F18016900205E0AD
:100B0000B4090512098F800A900205E0B40A0312A5
:100B10000BDE020A1B8F1A8E198D188C17851CA7E5
:100B2000AF1AAE19AD18AC1778081207298FF7E580
:100B30001AFF8FFB851BFC75F26E20AF3D75F30528
:100B4000E5A7651C703475F40AE51DB4552C75F5E0
:100B500009AF1AAE19AD18AC177808120729A80406
:100B6000A905AA06AB07AFF7E4FCFDFEC312071800
:100B7000700875F6060000000000E4F5A7228F1447
:100B80008E138D128C118515A7AF14AE13AD12AC58
:100B90001178081207298FF775F2E620AF3C75F33C
:100BA00005E5A76515703375F40AE51DB4552B7579
:100BB000F509AF14AE13AD12AC117808120729A8CD
:100BC00004A905AA06AB07AFF7E4FCFDFEC31207B4
:100BD00018700775F60600000000E4F5A722E490FF
:100BE0000206F0752C0A751D55F515FF7E0EFDFCED
:100BF000120B7EE4F515FF7E0EFDFC120C8C502AC4
:100C0000200130751B5AE4F51C7FFF7E0FFDFC129E
:100C10000B15E4F51B7FFF7E0FFDFC120D94EF64B6
:100C20005A6010900206740380059002067402F068
:100C3000E4F52CE4F51D2253B1F8120DACE4F51BDC
:100C40007FFF7E0FFDFC120D94EF645A7026C201E7
:100C5000751D55120D3850028005120D385005E4EF
:100C6000F51D8024E4F51D758E55438702000000B4
:100C7000000080F0E4F51B7FFF7E0FFDFC120D9459
:100C8000BFA505D2010200A6121000228F148E13F8
:100C90008D128C11D2048515A7E4F516F517AE1642
:100CA000AF17E4FCFDFB7A02F9F8D3120718401FD6
:100CB000E5172514FFE51635138F82F583E493605D
:100CC00004C204800A0517E51770D3051680CFE427
:100CD000F5A7A20422E4900206F0A3E0FFB4490FB6
:100CE000A3E0B4410AA3E0B45005C201D20022EF50
:100CF000B44911900208E0B4530AA3E0B45005D2FD
:100D000001D20022900206740AF0C200227580F817
:100D100075E18F75E9C875908075E27F75EA807519
:100D2000A0E075E33F75EBC075B01975E4E675ECAE
:100D3000194380C043E98022D20312077CEF701967
:100D4000F515FF7E0EFDFC120B7EE4F515FF7E0E01
:100D5000FDFC120C8C92038002C203A2032275C414
:100D600032E4F587759850759D7F759C64759E0477
:100D7000439D80759A0A759BFF2275817F75B20825
:100D8000000000000000000043B20478FFE4F6D841
:100D9000FD020C378F1A8E198D188C17E4851BA74E
:100DA000851A8285198393FFE4F5A722120DB512E7
:100DB0000D0DC20022E4F5A8F5A9F5AA2200000055
:100DC0000000000000000000000000000000000023
:100DD0000000000000000000000000000000000013
:100DE0000000000000000000000000000000000003
:100DF00000000000000000000000000000000000F3
:101C7A00021FC2E86480F8E933E83360110460F0B7
:101C8A00ED33EC337009E8FCE9FDEAFEEBFF2204D0
:101C9A0060DED3EB9FEA9EE99DE8C2E78CF0C2F7CB
:101CAA0095F0400CE8CCF8E9CDF9EACEFAEBCFFB97
:101CBA00121F8D85D0F05804700320D5B3E8047044
:101CCA00075002B2D5021FCC92D5EC0460F7E4CCDF
:101CDA00C0E0C398F8603B94186008400DD0E0FB60
:101CEA00021FA4E4FBFAC9FC8028E830E406E4C930
:101CFA00FBE4CAFCE830E305E4C9CACBFCE85407B4
:101D0A006010F8C3E913F9EA13FAEB13FBEC13FCBE
:101D1A00D8F130F52FC3E49CFCEF9BFFEE9AFEED61
:101D2A0099FDD0E0FBEF4E4D4C701222DB03021FEF
:101D3A00C9EC2CFCEF33FFEE33FEED33FDED30E75B
:101D4A00EB021FA4EF2BFFEE3AFEED39FDD0E0FBCC
:101D5A0050130BBB0003021FCCED13FDEE13FEEF75
:081D6A0013FFEC13FC021FA49F
:101D7200EC4D6011E8497017ED33EC3304600DE46B
:101D8200FCFFFEFD22E933E8330470F8021FC212A1
:101D92001F8D58046009E4CC2481500628500902A2
:101DA2001FCC284003021FC9C0E0EB4A7044B9802F
:101DB20006D0E0FB021FB8EF4E701CBD8008EBFF9F
:101DC200EAFEE9FD80EBE98DF0A4FEE5F0021E5B80
:101DD200E9CDF9EAFEEBFFEF89F0A4FCE5F0CE894C
:101DE200F0A42EFFE435F0CD89F0A42DFEE435F009
:101DF2008067EF4E7005BD80D780C3EF8BF0A4AC37
:101E0200F0EE8BF0A42CFCE435F0F8EF8AF0A42C71
:101E1200E5F038FCE433CB8DF0A42CFCE5F03BF884
:101E2200EE8AF0A42CFCE5F038F8E433CF89F0A474
:101E32002CFCE5F038CF3400CE89F0A42FFFE5F07A
:101E42003EFEE433C98DF0A42EFEE5F039CD8AF0D2
:101E5200A42FFFE5F03EFEE43DFD33D0E0FB50074A
:101E62000BBB000F021FCCEC2CFCEF33FFEE33FE5A
:061E7200ED33FD021FA488
:101E7800021FCCEC5D046005E859047003021FC220
:101E8800121F8D580460F6EC4860F2EC7004FDFEF9
:101E9800FF22C860DB2481C85009C398600250063D
:101EA800021FC99850CAF582E9294B4A7005AB82CE
:101EB800021FB875F0007C1A7880C3EF9BEE9AED8C
:101EC80099400DC3EF9BFFEE9AFEED99FDE842F0B5
:101ED800DC23ACF0D0E0FFD0E0FED0E0FDAB822008
:101EE800E7101BEB60BAEC2CFCEF33FFEE33FEED92
:101EF80033FD021FA4E803F830E705C0F075F000D1
:101F0800EF2FFFEE33FEED33FD40B830E7C280AA75
:101F180075F020800E75F010800575F0087D007E44
:101F2800007F003392D530D5031223A3EC33401041
:101F3800EF33FFEE33FEED33FDEC33FCD5F0ED224D
:0E1F4800E5F0247EA2D513CC92E7CDCEFF2289
:101F5600EDD2E7CD33EC3392D524814006E4FFFE83
:101F6600FDFC22FCE4CFCECDCC24E0501174FF80E2
:101F7600EDC3CC13CCCD13CDCE13CECF13CF04707F
:071F8600F030D5DE0223A3B9
:102C2300E51524BAF582E43402F583E00515229014
:102C330002B73054039002BAE475F0011224E6029D
:102C43002189204DE97F2ED24D8018EF540F249017
:102C5300D43440D4FF30510BEF24BFB41A005003D7
:102C63002461FFE516600215160519E519700205C2
:102C73001830540E9002B7E475F0011224E6EF0207
:102C830021CF027F517403D2548003E4C254F5155B
:102C93009002B71224FDE4F516F518F519E5166050
:102CA300077F20122C6680F57517FFC24EC24DC2F6
:102CB3004FC250C252C253C255122C32FF700D3054
:102CC30054057F00122C77AF19AE1822B4255FC2CA
:102CD300D5C251122C32FF24D0B40A00501A75F019
:102CE3000A781630D50508B6FF0106C6A426F620D5
:102CF300D5047002D25080D924CFB41A00EF500407
:102D0300C2E5D251022F69D24E80C6D24D80C0D2C5
:102D13004F80BCD2D580BAD25280B47F20122C66A9
:102D2300204F077401B5160040F1122C23FF122C1B
:102D330066022CA0D255D2538095122C23FB122C61
:102D430023FA122C23F94A4B700679677A307BFFFA
:102D5300204F2EE516602A7E008E82758300122195
:102D6300A260060EEE651770F0C2D5EBC0E0EAC0B4
:102D7300E0E9C0E0EE122FCAD0E0F9D0E0FAD0E0EB
:102D8300FB122189FF60AAEBC0E0EAC0E0E9C0E0E2
:102D9300122C66D0E02401F9D0E03400FAD0E0FB35
:102DA300E5170460DCD517D98087D24F80A2122F94
:102DB300AC60F7E517700104121FD7A917600DE582
:102DC30017600914F517123054EF60F3EA30E70285
:102DD300F404C3995079EAF425170430E701E404B5
:102DE300F517800D122FAC60C1EA05172517121FC6
:102DF300D7EA9002E6F030E701E4251704D517047B
:102E030020520114122FCAE4C0E01230549002E69B
:102E1300E0601320E70714F0122C4E802204F0D058
:102E2300E014C0E07F00122C4EE5176007122C451A
:102E33001517800B305203122C45D0E0022CA0D082
:102E4300E00480C4122FAC609EE51704121FD790D4
:102E530002E6EAF0E5172052026001042404122F6F
:012E6300CAA4
:102E640074FF04C0E0123054122C4EE517205202B5
:102E74006003122C45D0E0B517E87F45122C58901A
:102E840002E6E07F2B30E7047F2DF404C0E0122C2F
:102E940066D0E075F00A84C0F0122C4FD0E0122CFA
:102EA4004F022CA0791080027908C253C2558008C1
:102EB400D2D5790A8004790AC2D5E517047002F5DF
:102EC40017E4FAFDFEFF122C23FC7B08204E13129C
:102ED4002C23FD7B10304D0A122C23FE122C23FFD1
:102EE4007B20EC3382D592D55013C3E4304D069F3A
:102EF400FFE49EFEE4204E039DFDE49CFCE4CBF83D
:102F0400C24EEC700CCFCECDCCE824F8F870F38030
:102F140017C3EF33FFEE33FEED33FDEC33FCEB333D
:102F2400FB994002FB0FD8E9EB304E05F8D0E0C422
:102F340048B24EC0E00AEC4D4E4F78207B0070C280
:102F4400EAB5170040BCC0E0122FCCD0F0D0E0208E
:102F54004E04C4C0E0C4B24EC0F0122C4FD0F0D521
:102F6400F0EB022CA01225062D3D532EA8582D0E51
:102F74004C2D0A422EAC4F2EB4442EB4492D23437B
:102F84002EBA552DE7462E47452DB1473087502D93
:102F9400122D2D162E2D392B2D1A232D372030705E
:102FA4002A2CD24800002D31E517B4FF037517060B
:102FB400122C23FC122C23FD122C23FE122C23FF93
:102FC4009002DF022014790AA2D52050143052094D
:102FD400B910020404B9080104A2D5205302500117
:102FE40004204F68924FB516005034C0E07F203063
:102FF40050197F30A24F72537252500F123023C2B5
:103004004FC253C252C2557F30800F305203E9C0C1
:10301400E0122C66305203D0E0F9D0E0B516CC3083
:1030240052177F30B9100C122C667F583051077F2D
:10303400788003B90803122C66304F057F2D022CCB
:10304400667F202055F87F2B2053F322924F80CFA8
:103054007F00B40700500B24DFF582E43402F583CB
:10306400E0FF22286E756C6C2900D24E122C23309E
:103074004EF8C24E781630D50108F6022CD22D50E7
:10308400434958122C232403B405004001E4903032
:103094008293122C57743A122C57D250751604028C
:0230A4002EA854
:101F8D00E9D2E7C933E833F892D5EDD2E7CD33EC9A
:071F9D0033FC5002B2D52213
:101FA400EC30E7100FBF000C0EBE00080DBD00049E
:101FB4000BEB6014A2D5EB13FCED92E7FD2274FF4A
:101FC400FCFDFEFF22E480F8A2D574FF13FC7D80A3
:031FD400E480EFB7
:101FD700F920E73624F950037907E4F42402FBE5F6
:101FE70082158270021583DBF6E024FB501BE96043
:101FF70014E4F0E582158270021583E004F0B40A58
:0D20070008E4F0D9EE7401F00A22C2D522DF
:10201400ED33EC3392D5FA602AB4FF33EDC2E77B9B
:10202400FF60067A207939E4227A20794220D504A7
:102034007A20793D224E614E002B494E46002D49AF
:102044004E4600E47A08F0A3DAFC7B00740722C051
:1020540083C082ECC0E0EDC0E0EEC0E0EFC0E0EA97
:1020640075F010A4CAABF075F04DA42BFBE435F069
:10207400FCEA2410FAEB34C5FBEC34D9FCEDC2E7DE
:10208400FF75F056A4F42411C5F0F434C58FF0A400
:102094002AE5F03BE43CF020E714122149D0E0FFAC
:1020A400D0E0FED0E0FDD0E0FC121E7B8014F404EE
:1020B400122149D0E0FFD0E0FED0E0FDD0E0FC12D8
:1020C4001D72D082D083E0FAEDD2E7CD33EC332415
:1020D40082FBE4C3CF33CFCE33CECD33CD33DBF36A
:1020E4007B0775F00A846004F0A31B0AE5F0F0A3F3
:1020F4008FF0740AA4FFACF08EF0740AA42CFEAC2A
:10210400F050010C8DF0740AA42CFDE435F0F0A31A
:05211400DBDE74072270
:102119003F8000004120000042C80000447A0000CE
:10212900461C400047C35000497424004B18968050
:102139004CBEBC205A0E1BCA6753C21C749DC5AE47
:10214900FB60065407601C2323122177EB54386087
:1021590009122163122172121D72ECF8EDF9EEFADF
:10216900EFCB22EB12217280F1543803241C902109
:1021790019FE93FC0EEE93FD0EEE930ECE93FF2205
:10218900BB010689828A83E0225002E722BBFE0254
:09219900E32289828A83E4932287
:1021A200BB010CE58229F582E5833AF583E02250F2
:1021B20006E92582F8E622BBFE06E92582F8E2223C
:0D21C200E58229F582E5833AF583E4932256
:1021CF00BB010689828A83F0225002F722BBFE01EF
:0221DF00F322E9
:1021E100EF8DF0A4A8F0CF8CF0A428CE8DF0A42E12
:0221F100FE22CC
:1021F300BC000BBE0029EF8DF084FFADF022E4CCD0
:10220300F875F008EF2FFFEE33FEEC33FCEE9DEC98
:10221300984005FCEE9DFE0FD5F0E9E4CEFD22EDDE
:10222300F8F5F0EE8420D21CFEADF075F008EF2F28
:10223300FFED33FD4007985006D5F0F222C398FD19
:052243000FD5F0EA22B6
:10224800C5F0F8A3E028F0C5F0F8E5821582700221
:062258001583E038F022BE
:0D225E00EF2BFFEE3AFEED39FDEC38FC22CF
:0E226B00C3EF9BFFEE9AFEED99FDEC98FC226E
:10227900E88FF0A4CC8BF0A42CFCE98EF0A42CFC04
:102289008AF0EDA42CFCEA8EF0A4CDA8F08BF0A482
:102299002DCC3825F0FDE98FF0A42CCD35F0FCEBE1
:1022A9008EF0A4FEA9F0EB8FF0A4CFC5F02ECD39A6
:0F22B900FEE43CFCEAA42DCE35F0FDE43CFC2213
:1022C80075F008758200EF2FFFEE33FECD33CDCCCD
:1022D80033CCC58233C5829BED9AEC99E582984050
:1022E8000CF582EE9BFEED9AFDEC99FC0FD5F0D62D
:1022F800E4CEFBE4CDFAE4CCF9A88222B800C1B957
:102308000059BA002DEC8BF084CFCECDFCE5F0CB94
:10231800F97818EF2FFFEE33FEED33FDEC33FCEBCD
:1023280033FB10D703994004EB99FB0FD8E5E4F988
:10233800FA227818EF2FFFEE33FEED33FDEC33FC75
:10234800C933C910D7059BE99A4007EC9BFCE99A69
:10235800F90FD8E0E4C9FAE4CCFB2275F010EF2FAE
:10236800FFEE33FEED33FDCC33CCC833C810D707AE
:102378009BEC9AE899400AED9BFDEC9AFCE899F8E9
:0E2388000FD5F0DAE4CDFBE4CCFAE4C8F9227C
:10760200C2D5E830E70FB2D5E4C39BFBE49AFAE4B3
:1076120099F9E498F8EC30E717B2D51276381223CC
:1076220004E4C39BFBE49AFAE499F9E498F8800332
:1076320012230430D50DE4C39FFFE49EFEE49DFDBA
:04764200E49CFC22A6
:0D239600EF4BFFEE4AFEED49FDEC48FC2246
:0E23A300C3E49FFFE49EFEE49DFDE49CFC224B
:1023B100EB9FF5F0EA9E42F0E99D42F0EC6480C8A3
:0623C10064809845F02243
:1023C700EB9FF5F0EA9E42F0E99D42F0E89C45F06C
:0123D70022E3
:1023D800E8600FECC313FCED13FDEE13FEEF13FFE3
:0323E800D8F12207
:1023EB00E86010ECA2E713FCED13FDEE13FEEF1308
:0423FB00FFD8F022F5
:1023FF00E8600FEFC333FFEE33FEED33FDEC33FC3C
:03240F00D8F122DF
:0C241200E6FC08E6FD08E6FE08E6FF22F6
:0C241E00E0FCA3E0FDA3E0FEA3E0FF2231
:0D242A00E6FB08E6F908E6FA08E6CBF82222
:0C243700E0F8A3E0F9A3E0FAA3E0FB2228
:102443007401FF3395E0FEFDFCA3A3A3E02FFFF08F
:10245300E582158270021583E03EFEF0E582158267
:1024630070021583E03DFDF0E5821582700215834D
:05247300E03CFCF0223A
:0C247800ECF608EDF608EEF608EFF62290
:0C248400ECF0A3EDF0A3EEF0A3EFF022CB
:10249000D083D082E493F608740193F60874029313
:0924A000F608740393F67404734A
:1024A900A8828583F0D083D0821224C01224C0125E
:1024B90024C01224C0E473E493A3C583C5F0C58383
:1024C900C8C582C8F0A3C583C5F0C583C8C582C87D
:0124D90022E0
:0C24DA00A42582F582E5F03583F583220D
:1024E600F8E0FBA3A3E0F925F0F0E582158270027F
:0724F6001583E0FA38F02223
:0924FD00EBF0A3EAF0A3E9F022E0
:10250600D083D082F8E4937012740193700DA3A364
:1025160093F8740193F5828883E473740293686078
:06252600EFA3A3A380DF78
:10252C00EC8EF0A4CCC5F0CCCDF8EFA4CEC5F02D3C
:10253C00FDE43CFCE8A42EC8C5F03DFDE43CFCEFFA
:0D254C00A4FFE5F028FEE43DFDE43CFC2288
:00000001FF
